:020000040800F2
:10500000F81B0020D5500008CD8B0008DD82000879
:105010000000000000000000000000000000000090
:105020000000000000000000000000000D9A0008D1
:1050300000000000000000008D930008499B00085C
:10504000E7500008E7500008E7500008E750000864
:10505000E7500008D95C0008E7500008E750000856
:1050600000000000E7500008015C0008E75000085D
:10507000E7500008BD87000800000000E750000866
:1050800000000000E75000080000000000000000E1
:10509000E750000800000000E7500008E750000853
:1050A000E7500008E7500008E7500008C5A50008D1
:1050B000E7500008E7500008000000000000000072
:1050C0000348854600F0E8FC0048004739B900086D
:1050D000F81B00200448804704480047FEE7FEE72D
:1050E000FEE7FEE7FEE7FEE7E59B0008C15000088B
:1050F00030B50B46014600202022012409E00D4670
:10510000D5409D4205D31D469540491B25469540F7
:1051100040191546521E002DF1DC30BDF0B51FB40C
:105120000646002082B005464024019100901BE015
:10513000019922460F46304600F098FB049A059BE1
:10514000801A994110D310461946224600F07EFB82
:10515000361A8F410197224601200021009F00F05E
:1051600075FB38184D4100902046641E0028DFDC96
:10517000019B00982946324607B0F0BD03460B4319
:105180009B0703D009E008C9121F08C0042AFAD2FD
:1051900003E00B780370401C491C521EF9D2704783
:1051A000D2B201E00270401C491EFBD270470022BF
:1051B000F6E710B513460A4604461946FFF7F0FF16
:1051C000204610BD30B504460020034600E05B1CBD
:1051D000934203D2E05CCD5C401BF8D030BDF8B503
:1051E00002464A40D40F42004B0052085B089A42E4
:1051F00002D20246084611464A0023D0C30D4A0097
:10520000DDB2120EAD1A202D35DA49020126490A07
:10521000F6058A19002C00D0524220214F1B11465E
:10522000B9402A411018C20D9A4221D0002C17D043
:10523000012D08DCDA05801AD20F8019D207DBB203
:1052400000F040FBF8BDDA05801A012340001B0680
:10525000C01880185A428018CA0F1043490007E04E
:105260004908C2071143DA05801A801940088018DE
:1052700000F020FBF8BD61000122511A001BF7E786
:105280000122D2075140AAE70122D2075040A6E7E7
:1052900070B502464A40D50F40004A00ED0740086D
:1052A0005208002814D0002A12D0C40DD30D410298
:1052B0000120C0055202490A520AE41A09181218BC
:1052C0007D34914201D3641C00E04900002C01DAD6
:1052D000002070BD0023914201D3891A0343400886
:1052E00049000028F7D100290AD0914202D10121BA
:1052F000C90705E0914201D2012101E00121C94322
:10530000E005C018401900F0D5FA70BD420005D084
:105310004200120E52428A4201DB00207047C9054A
:1053200008187047F0B507460846584087B0C00FC8
:10533000049048000E46590040084908BC1A8841AC
:1053400005D2384631461E4617460B4602465800DF
:10535000400810434CD0300D039040055900400DDB
:10536000490D0590401A0290402872DA1803012175
:10537000000B09050843019004980092002805D00D
:1053800001995242002088410092019002984021E8
:105390000A1A0199009800F059FA05460C466B4626
:1053A00007CB00F074FAC0197141039A0E0D002367
:1053B000D71756401A467A40164344D0049A002A1A
:1053C0002DD0029A012A039A15DC1205C01A9141C8
:1053D00001263605001C7141D20F059ED2070093AD
:1053E000019202962A46234600F0B2FA07B0F0BDB9
:1053F00038463146FAE71605224A0F46B218C01A57
:10540000B74101210905001C4F4100187F41114699
:1054100018187941E20F10436D19644113E0E20757
:105420006D0815436408C2071443039A0126120548
:10543000C01A91413605001C7141CE074008304327
:105440004908C01851412A46234600F074FACDE7B6
:10545000FFE7049801224000C117121A00238B4174
:1054600004983146C417381AA141EEE730B401243C
:10547000E407634030BC55E730B40124E4076140E1
:1054800030BC4FE70000E0FFF0B51FB488B00B99C7
:105490000998002448400999C00F4900490809911A
:1054A000C0070B990090490049080B910999089889
:1054B000A64608431CD00B990A98084318D00998AF
:1054C00001244000420D4800410D099824050003C5
:1054D000000B204309900B980003000B20430B9016
:1054E00050181C494018002201901446104605E04F
:1054F000002001460DB0F0BD032801DA034600E0AC
:1055000003239C46C11A0AAE0AE05F0008ADED5BBA
:105510004F00F75B7D430027AA187C41491C5B1EA6
:105520006145F2DD410004AB5A522104120C0A43DA
:10553000240C401C0828DFDB01980290009970467B
:1055400001910090059B049A0799069800F000FAD3
:10555000D0E700000DFCFFFFF0B50C465C4085B0C5
:10556000E40FE40703944C000026640859009446B5
:10557000490802460296224321D062460A431ED0C1
:105580006200570D4A000E032303550D0124024605
:105590002C492405781B1B0B360B4018234326434C
:1055A000614600901C46501AB44103D30098401C39
:1055B000009002E0921800985B41002803DA002076
:1055C000014605B0F0BD00200121090507468646C9
:1055D00011E064461D46141BB54106D36546521BB7
:1055E000B341744607430C43A646CD07400849081B
:1055F000284392185B4105460D43EAD110461843F3
:1056000013D06046194650407140084306D06046AA
:10561000101AB34106D20122002306E00022012322
:10562000DB0702E00122D2435310009874460105C3
:10563000381C6141029C039D0019694100F07BF90F
:10564000BFE70000FD03000070B54B005B0803439B
:105650000BD04B005C0D002633466542B341D41796
:10566000AD1AA34102DB0020014670BD12053018BF
:10567000514170BDC217C10F504010B54018CA0744
:105680009623002100F01EF910BD10B500229623CC
:10569000114600F017F910BD0EB5C217C10F5040EA
:1056A000CA0740180021054B0293019200910A4657
:1056B0000B4600F04DF903B000BD000033040000BC
:1056C0000EB505490291002100910A460B46019151
:1056D00000F03EF903B000BD330400004100400279
:1056E0000122400AD205090E80187F2901DA002024
:1056F0007047962903DC9622511AC84070479639A4
:105700008840704770B5CD0F4A0009030123090B8B
:105710001B0519430B4BED070024520D9A4201DA89
:10572000002070BD074B34339A4203DC9A1A00F014
:105730009DF802E00449511888402C43F1D04042C2
:1057400070BD0000FF030000CDFBFFFF4A0009030E
:105750000123090B1B051943094B10B5520D9A4241
:1057600001DA002010BD064B34339A4203DC9A1A4A
:1057700000F07CF810BD03495118884010BD0000AE
:10578000FF030000CDFBFFFFC20FD207400040081F
:105790000BD0C10D0723DB01C91840020905400ADF
:1057A0001143C2084007114370470020014670476B
:1057B00010B5002904DB0124E40740428C41214656
:1057C000002B04DB1C460123DB075242A3418B4222
:1057D00000D1824210BD000010B5002904DB012475
:1057E000E40740428C412146002B04DB1C46012388
:1057F000DB075242A341994200D1904210BD000004
:10580000CB0FDB07490010B5490802460A4307D011
:105810000A0D07240903E401090B121B002A01DC0D
:10582000002010BDC900440F0C43C100E018D20590
:10583000801800F03FF810BD0122D207002800DBDD
:10584000101A002900DB511A8142704710B5202A36
:1058500004DB0146203A9140002010BD91402023F6
:105860009C1A0346E3401943904010BD10B5202A0E
:1058700004DB0846203AD040002110BD0B46D3403F
:10588000D0402024A21A91400843194610BD10B5FB
:10589000202A06DBCB170846203A1041C1170B43DC
:1058A00006E00B461341D0402024A21A9140084341
:1058B000194610BD002904DA401C490001D14008F6
:1058C0004000704770B40024050C05D1102400047A
:1058D00002D1002921D01124050E01D10002083483
:1058E000050F01D10001241D850F01D18000A41CEA
:1058F000002801DB4000641C002908D020252E1B55
:105900000D46F540A14000D001212943084301067E
:105910001B1B000ADB1D02D5002070BC7047DB0595
:10592000181880180029F8DA401C4900F5D170BC1D
:1059300040084000704710B5002B08DA0024401CD6
:10594000614192185B411A4301D14008400010BDEB
:10595000F0B51FB482B005460C0003D0084604F031
:10596000E5FE02E004F0E2FE20300246009021460F
:105970002846FFF76BFF049B059A04460F46184321
:105980001143084314D0184610431BD000984021FF
:105990000A1A18460599FFF769FF05460E46009A50
:1059A00005990498FFF752FF084305D0012004E051
:1059B0002046394607B0F0BD0020C11705430E430D
:1059C0002C43374300990E986305401A7905E40A81
:1059D00000220C43FD0A0A3002D500200146E9E707
:1059E0000105101969410C9C0D9D00196941FFF7D3
:1059F000A2FFDFE7FEB500231A461B1A8A4103DB2C
:105A00000020014603B0F0BD4A000D0301212D0B1B
:105A10000905520D0D43D10702D100186D41521EE8
:105A20005110FF31FF310131002704463E46384610
:105A3000009701910246012100200905FFF716FF9A
:105A4000C3197141F818324684468E464A41614670
:105A50002846611A904104D36046241A954176463F
:105A60001F46241900986D41401C00903428E1DD48
:105A7000F91930467041091BA84103D20022D243D4
:105A8000134601E00022134601980105381C7141BC
:105A9000FFF751FFB6E70000064C0125064E05E072
:105AA000E36807CC2B430C3C98471034B442F7D33F
:105AB000FFF70AFB18C8000838C8000870B58C1832
:105AC0000578401C6B075B0F01D10378401C2A113D
:105AD00006D10278401C03E006780E70401C491C79
:105AE0005B1EF9D12B0705D40023521E0DD40B7079
:105AF000491CFAE70378401CCB1A921C03E01D787E
:105B00000D70491C5B1C521EF9D5A142D8D3002050
:105B100070BD000038B50446064805490068FFF727
:105B2000E7FA604300E0401E00900028FBD138BD3A
:105B300040420F0084010020F8B5044600688168E7
:105B40008907890F012902D10168C90722D181681B
:105B5000114A10261140012500290ED181682943E0
:105B600081600120FFF7D6FF01F026F807460CE020
:105B700001F022F8C01B0A2807D9606D3043606528
:105B8000A06D2843A0650120F8BD20680068C043CF
:105B9000C007EDD10020F8BD170000801FB50B48ED
:105BA00000900B4801900B4802900B480390694607
:105BB0000A4805F0B1F90A4A08481146083905F0C3
:105BC00099F800F06DFA002004B010BD25C6000859
:105BD00001C6000861C600085FC6000890010020E9
:105BE0001000002010B500231A4603E0845CE3187F
:105BF0009BB2521C8A42F9D3D84380B210BD000038
:105C000010B5034800F094FD024800F091FD10BD6E
:105C1000981700205017002030B5446C1C252C40EC
:105C20000125A540046C6560046863608368102BDF
:105C3000036803D099600068C26030BD9A60006854
:105C4000C16030BD1449012048720A4602205E320C
:105C5000507203203C3A507204200E3A50720F48A2
:105C60000D4B0078087022310870203108770C49FC
:105C70005A1C0878587149789971233318715971F1
:105C8000203318775977107551751A461E321075E2
:105C90005175107651767047E81100203E010020C2
:105CA0006001002010B503F087FE202003F042FFC2
:105CB000012005F09BFB002003F03CFF044805F0A9
:105CC00039FA044805F0E8FC002005F01DFD10BD80
:105CD0000001002083800000F8B5052001210007A5
:105CE00000F056FF0025144C002800D06560134ECC
:105CF0000221304600F04CFF002815D10120207011
:105D00000F48808F00280ED00127BF02002239469D
:105D1000304600F04AFF0A2004F05CFF01223946B9
:105D2000304600F042FF6560012000F069FE02206D
:105D300000F066FEF8BD0000700100200004005075
:105D4000E80D00207047000010B5084900224A61A4
:105D500007494B684C1523434B604B680824234389
:105D60004B60C009C001026010BD0000E0170020B8
:105D7000002002407FB500250C460646039500F042
:105D80000FFEE009029003A901960095684600F015
:105D90009FFD002804D000F0D7FD002004B070BDA6
:105DA00000F0D2FD0120F9E710B5002302E0C45C49
:105DB000CC545B1C9342FAD310BD000010B5214AAD
:105DC00000219069C305204804D541690223194385
:105DD0004161911593699B0505D5436901242343CE
:105DE00043616302194393695B0505D54369082440
:105DF00023434361E301194393691B0505D54369B7
:105E00000424234343616302194393699B0405D52A
:105E100043691024234343616302194393699B033D
:105E200004D5446920231C43446119439369DB036F
:105E300005D54369402423434361A0020143916196
:105E400010BD000000200240E017002070B505469C
:105E500000F0B2FE0646184C0AE0681C08D0002D7F
:105E600004D000F0A9FE801BA84201D9032070BD18
:105E7000A069C007F1D1A069800701D50220A06107
:105E8000A069C00511D4A06980050ED4A0694005A1
:105E90000BD4A069000508D4A069800405D4A069CA
:105EA000800302D4A069C00303D5FFF787FF012058
:105EB00070BD002070BD000000200240F8B51746FC
:105EC000002605460C4600F06BFD09E0294602203D
:105ED000226800F047FD002804D1241D2D1D361D29
:105EE000BE42F3D300F030FDBE4201D20020F8BD27
:105EF0000120F8BD10B5084902460020054B49793C
:105F000005E044001C5B944203D0401CC0B28842B0
:105F1000F7D310BD8C1300207000002010B500F0E6
:105F20003CFE10BD10B5094801F05CF880B2FFF7E7
:105F3000C7FB074A074BFFF7A7FA0022064BFFF7FC
:105F40000BFBFFF703FC80B210BD0000041600201D
:105F5000F853E3A59B843E4000408F4070B5002479
:105F6000204603F0ADF947494748A200641CE4B25B
:105F70008150142CF9D3464944480A78027549786F
:105F8000417544490A780276497841763F490520AF
:105F9000133148720A2005F06FFB7D20400105F0A7
:105FA00085FB3A49002213310C2005F04FFC0021FB
:105FB0000C2005F05DFC384801F014F8344C012544
:105FC000223CA084AD0309E0334801F00BF880B215
:105FD000A084618EFF392D39884206DB618E80B244
:105FE0008842F1D349198842EED8022005F094FB8B
:105FF000002003F065F9294D00210F2005F0BCFABF
:106000002842E063F8D0E06B411C38D0400435D51D
:106010008122D20100210F2005F0EDFB002110208C
:1060200005F0AAFA41061948490E0022C73005F0CA
:10603000D9FA164DC735687A05281FD102221549AD
:10604000681DFFF7BFF8002818D11148AE7C6671B3
:106050000422691C3230FFF791F8294613310846B3
:1060600072000D466930FFF789F8607929464200D1
:1060700005484838FFF782F80320207070BD04F00F
:10608000C9FB0000FFFF0100EC13002049120020B3
:1060900092000020600100200416002000D0272478
:1060A00010B5144C1448224610321146083904F039
:1060B00021FE0022114BE168A068FFF74DFA104A5B
:1060C000104B05F03FFD00220F4BFFF7D5F90022E2
:1060D0000E4BFFF7D9F9FFF793FB20600022134620
:1060E000E168A068FFF764FB01D0206810BD0020C4
:1060F000206010BD000000209001002000AA8F4009
:106100006C45D9CC955BC83F0000F03F40A5E54009
:1061100010B5084800F096FA0A21064800F032FA55
:10612000044800F01DF9800503D5024800F01AF973
:1061300080B210BDA8150020F8B52F4D0022012116
:10614000284600F032FDFFF7E3FFFFF79EFA2B4EE3
:106150003146FFF79DF82A4C0122A06011462846DF
:1061600000F023FD2749A068002588423EDB207807
:10617000254F002815D02570FFF7CAFFFFF785FAD5
:106180003146FFF785F8A060FFF7FEFA00223B4694
:10619000FFF76CF900221D4BFFF776F9FFF730FB94
:1061A0006060A068FFF7F0FA00223B46FFF75EF957
:1061B000174A184BFFF768F906460F466068FFF765
:1061C000E3FA134A144B5242FFF75EF932463B465C
:1061D000FFF7A8F8FFF714FB10496060884201DD63
:1061E000616004E0FF21C905C84200D365606068B2
:1061F000FFF774FAC0B2F8BD0004005000401B4421
:10620000480000200000604000000C4000E06440B6
:106210003333333333B33040CCCCEC3F0000C8428F
:10622000F8B5054604464035287C0026012808D0EC
:1062300001202874206881688907890F01290ED1FF
:1062400001E00220F8BD0168C90708D0606D202177
:10625000084360650126002028743046F8BD616D52
:10626000FF2201329143022211436165C16889070F
:10627000890F0091C16889088900C1602068816820
:1062800092071143816000F097FC07460EE000F092
:1062900093FCC01B0A2809D9606D02218843102194
:1062A00008436065002028740120F8BD20688068DC
:1062B0000028ECDB2068C168009A1143C160606D62
:1062C00080088000401C6065C5E70000F8B5064600
:1062D0000D464036317C01290DD001213174016811
:1062E0008A68520709D5416D20221143416500207B
:1062F00030740120F8BD0220F8BD174B6A68D8053C
:1063000047109A42154C8A6A2B6812D05B035B0BCC
:106310001A438A622968490305D5A1680143A1602F
:106320000A20FFF7F7FB2868800312D5A0683843DE
:106330000EE05B035B0B9A438A622968490302D52E
:10634000A1688143A1602868800302D5A068B84392
:10635000A06000203074F8BD01100000002701404B
:10636000406D70470068006C7047000070B5040015
:1063700006D0606D264600254036002802D006E093
:10638000012070BDA5653574204600F0D3F8606D1E
:10639000C00603D421688868400705D5606D1021C8
:1063A000084360653574EBE7606DFF22013290436E
:1063B00002221043606588688207920F5B48012AB9
:1063C00002D10A68D2072BD1032362689B079A4245
:1063D00005D05B429A4202D05B009A4209D10A6919
:1063E000920092080A6121680A6963681A430A6187
:1063F0000CE00A69920092080A6181680F229204F7
:106400009143816081686268114381602168CA6834
:1064100018239A43CA602168CA68A3681A43CA60ED
:10642000816801225206914381608168A28E5206E2
:106430001143816020688168C90004D48168012209
:106440001207114381602068C168394A1140C16058
:106450002069E168022825D0002001432046203031
:106460000278037B52035B001A431143226B1143F2
:10647000A26992031143E269D20311432268D368EF
:106480001943D160616A0A46FF3AC23A05D0A26A4E
:1064900011432268D3681943D16042780121012A4F
:1064A00002D00BE00420D8E70078002823D0606DEC
:1064B000202210436065A06D0843A065E06B0128B1
:1064C00020681FD00169C90703D001694908490044
:1064D000016120684169C908C900416120684169BA
:1064E000A26B11434161A565606D80088000401C6E
:1064F0006065002070BD2068C26801231B041A4338
:10650000C260DBE70269FF239B009A4302612068B7
:106510000269236CA66C1A43636C33431A4302610D
:10652000206802690A430261D3E7000000270140A6
:106530001902FEFF10B586B0044614216846FEF726
:1065400036FE0E492068884216D10D48416B42152F
:1065500011434163C16A01221143C162C06A6946A5
:10656000104005900220009003200190002002902E
:106570000520000700F050FA06B010BD00240140CD
:1065800000100240F8B504464069254640350E46E5
:1065900008280BD02068C068C00709D0606D202192
:1065A00008436065002028740120F8BD082700E03A
:1065B0000C2700F001FB009011E0701C0FD0002EA2
:1065C00005D000F0F9FA0099401AB04207D9606D81
:1065D000042108436065002028740320F8BD20686A
:1065E00000683842E9D0606D0121490208436065C6
:1065F0002068C16809058A0F0C21002A1BD12022BE
:10660000125D002A17D10268120714D58268530759
:106610000122002B08DB43688B434360606D13024B
:1066200098431043606506E0606D20231843606561
:10663000A06D1043A065A069002801D12068016009
:106640000020F8BD70B5044621680020896849071C
:1066500021D425464035297C01291CD001212974EB
:10666000E169012904D02046FFF766FA002811D11C
:10667000616D0A4A1140FF22013211436165002118
:10668000A165297422681C21116021688A6804238D
:106690001A438A6070BD022070BD0000FEF1FFFF4A
:1066A00030B5014620314A790023022A04D0042261
:1066B000C2630B71012030BD026814680E25AC4323
:1066C000146002681468640864001460446C1C223E
:1066D000144001221546006CA54045604A711846D9
:1066E0000B7130BD70B50024014620314A79022A71
:1066F00003D00421C163012418E0026813680E2549
:10670000AB431360026813685B085B001360436C63
:106710001C221340012215469D40036C5D604A71A6
:1067200000220A71816B002900D08847204670BD85
:10673000F0B4016C0D6801680C68466C1C230422DF
:106740001E401746B7402F420ED067070CD50C6885
:10675000A40602D40C6894430C60416C19408A4032
:10676000016C4A60016B1AE00227B74002462F40D5
:106770002032002F17D0A70715D50C68A40605D422
:106780000C680A25AC430C6001215171446C022154
:106790001C40036CA140596000211171C16A00299D
:1067A00018D0F0BC08470827B7402F4212D0240762
:1067B00010D50C680E25AC430C60446C01211C40C4
:1067C0000B46A340046C6360C163517100211171D9
:1067D000416BE4E7F0BC704770B504003CD01F4843
:1067E000256814212818FEF783FC800060641C488B
:1067F0002064022120462030024641712968194850
:10680000E3680140A068666918432369334318436D
:10681000A3691843E3691843236A184308432860AF
:106820000121A0688903884210D00D488030836A16
:10683000656C1C210D400F26AE40B3438362656C2E
:1068400063680D40816AAB400B4383620020E063C4
:1068500001215171107170BD012070BDF8FFFDBFA5
:10686000000002400F80FFFFF8B504468C46203040
:1068700001790025012909D00126067141790027F7
:10688000012905D0077102252846F8BD0220F8BD70
:1068900002214171E76320680168490849000160ED
:1068A00061462046FFF7B8F9206B00282068016890
:1068B00001D00E2205E004229143016020680168A6
:1068C0000A22114301602068016831430160DBE75F
:1068D000F8B51A4E0546307C0F46012807D0012036
:1068E00030741748FFF7B2FA010002D021E002200D
:1068F000F8BD0020C04338606C6814E02046FFF704
:1069000023FA0F48FFF7A2FA01460E48426808230F
:106910009A434260426843159A434260002901D07D
:106920003C6006E08034A8686A68C0018018A04214
:10693000E4D8002030740846F8BD0000E0170020BD
:1069400050C3000000200240054841680222114364
:1069500041604168012211434160002070470000FE
:1069600000200240F8B50C4C1646207C0F4601284A
:1069700008D0012020740948FFF768FA0025002894
:1069800002D006E00220F8BD65613E600348FFF7D3
:106990005DFA2574F8BD0000E017002050C3000028
:1069A00011484168C9070BD0EFF3108172B60F4A46
:1069B000C2600F4AC26081F310884168C9070ED1D6
:1069C000416889070DD5EFF3108172B6094A02615B
:1069D000094A026181F310884068800701D50120CF
:1069E000704700207047000000200240EFCDAB89C7
:1069F00005040302BFAE9D8C1615141370470000EA
:106A000010B504494A69024202D04861FFF7F6FF17
:106A100010BD000000040140FCB500230124A2E0E9
:106A200027462A469F403A406FD04D68012D05D039
:106A3000022D03D0112D01D0122D16D18568032609
:106A4000AC465D00AE46AE406546B543AC46CE684A
:106A50007546AE4065462E43866046680D79BE4356
:106A6000ED06ED0F9D4035434560C6685F00032588
:106A7000BD40AE46AE4335468E68BE402E43C6602E
:106A80004E68022E01D0122E14D1DE08B600361840
:106A90000196366A5D07B446EE0E0F25B5400096A6
:106AA0006646AE43B4460D69009EB54066462E4329
:106AB000019D2E6206687546AE430D79AD07AD0F98
:106AC000BD40354305604D68ED004BD5294D6E6BDB
:106AD00026436E639E08284DB6007519AC46AD6816
:106AE0009E07360F0F27B740BD4305273F07B84223
:106AF00001D1002715E0214FB84201D1012710E054
:106B00001F4FB84202D102270BE02BE01D4FB842C5
:106B100001D1032705E01C4FB84201D1052700E051
:106B20000627B7402F436546AF60184D2E684F6863
:106B30009643FF0300D516432E606E684F68964358
:106B4000BF0300D516436E60AE684F689643FF02E0
:106B500000D51643AE60EE684F689643BF0200D57D
:106B60001643EE605B1C0A681546DA4000D057E712
:106B7000FCBD000000100240000001400004005075
:106B800000080050000C0050001C005000040140A0
:106B90000069084000D001207047426913460B404D
:106BA0001B0491430B4383617047002A01D081612C
:106BB000704781627047000001488068704700009C
:106BC0007801002002488168027889188160704746
:106BD0007801002010B508480024016840221143C4
:106BE0000160204600F00AF8002801D0012401E0ED
:106BF00000F042FA204610BD0020024070B5044665
:106C00000D4D7D202978C000FEF772FA01460B4831
:106C10000068FEF76DFA00F02BFF002809D1042C64
:106C200007D200222146401E00F04EFA00206C6080
:106C300070BD012070BD000078010020840100209B
:106C400070477047F8B502F083FF604C0120E07098
:106C5000208AFEF71AFD01467F20C005FEF718FBCB
:106C60005B4D06462968FEF7BAFA28600120A16A42
:106C7000C005814201DA084603E03046FEF704FB16
:106C8000A062FF21C9050025C84200D3A562607833
:106C900000280BD102214F48FFF77AFF02004E492E
:106CA0004E4817D00022FFF780FFE56202214948D5
:106CB000FFF76EFF4A4E002855D0E562B08AFEF716
:106CC000E4FC434F3968FEF7B7FD5FD24549012028
:106CD00008705DE00122D1034048FFF766FF208A7B
:106CE000FEF7D3FC01467F20C005FEF7D1FAE16A2A
:106CF000FEF775FA3C49E0628842D7DD3848012743
:106D0000F926403000900A213046FEF7F1F90029BB
:106D100003D131493148FFF701F902212D48FFF72E
:106D200037FF002801D0002701E0002F12D10221F7
:106D30002848FFF72DFF00280CD104F0CBFE009966
:106D40000120888005F022FC642003F043FF2849DD
:106D50002648C8600A2003F03DFF3046761EF6B292
:106D60000028D0D1A2E7208AFEF78FFC01467F20C1
:106D7000C005FEF78DFAE16AFEF731FA1D49E062BF
:106D800088429BDB1A491948C86097E71548057087
:106D9000708F401EFEF76EFC3968FEF74DFD06D879
:106DA0002079002803D014490120087001E012481E
:106DB0000570708FFEF769FC3968FEF73DFD04D25F
:106DC0002079002801D004F049FEF8BD3C010020E4
:106DD00074010020000400500080000000000050FA
:106DE000E80D002076000020000040400400FA0575
:106DF00000ED00E00000A04083000020704770B567
:106E0000040010D0022025462035A873204601F04A
:106E1000DDFCA87B032805D0204600F0B9F800204F
:106E2000A873687370BD012070BD7047704710B5BE
:106E3000044600680168C943C90708D18168C9438D
:106E4000C90704D1012141602046FFF7FBFE2068FD
:106E50000168C943890708D48168C943890704D4F4
:106E6000022141602046FFF7EBFE20680168C9431C
:106E7000490708D48168C943490704D40421416003
:106E8000204600F0F7F820680168C943090708D4D4
:106E90008168C943090704D4082141602046FFF7EF
:106EA000ADFF20680168C943C90608D48168C94399
:106EB000C90604D4102141602046FFF7C2FE2068B5
:106EC0000168C943890608D48168C943890604D486
:106ED000202141602046FFF7A9FF20680168C943CF
:106EE000490608D48168C943490604D44021416059
:106EF0002046FFF79AFF10BDF8B5040005D02546DF
:106F00002035A87B002802D006E00120F8BD002033
:106F10006873204600F04EF80220A8732068C2680B
:106F200084466368012B01D10620824316486169BB
:106F3000814202D0072040038243002B01D1D82098
:106F400082431248A668024018463043676A266AA0
:106F50003E433043A66A30431043002B02D0012B3E
:106F600004D005E02369E2691A4300E0E2681043B7
:106F7000054A914202D0A269114308436146C860A4
:106F80000120A8730020F8BDFFFF0000F8F119FFF1
:106F900010B500680549884207D10548816B490052
:106FA000490881630D2000F073F810BD007C00409B
:106FB0000010024010B50068084988420CD108480A
:106FC000816BC20411438163002201210D2000F076
:106FD0007BF80D2000F06CF810BD0000007C004034
:106FE000001002400068C06970470000F8B5044610
:106FF0000220254620351746A8731D480268C304A1
:107000001A4302602068C2689B121A43C26020685B
:107010000269012632430261226810205060206814
:1070200081611021204601F041FC03281FD0216816
:1070300008204860206847610821204601F036FC9E
:10704000032814D0204601F0C1FBA87B03280ED0F2
:1070500020688168314381602068016931430161A2
:1070600020680169042211430161AE730020F8BD5C
:1070700000040140704700000448416B01221143A5
:107080004163816B02041143816370470010024029
:10709000002809DBC106C90E0120884003490860A9
:1070A000BFF34F8FBFF36F8F7047000080E100E0A8
:1070B000002805DBC106C90E01208840014908608F
:1070C0007047000000E100E010B503F081FB10BD47
:1070D00002494A6882434A607047000000700040DD
:1070E000024801688215114301607047007000403A
:1070F00002494A6802434A6070470000007000403D
:107100000548016802221143016004480169042214
:107110001143016130BF70470070004000ED00E096
:10712000F0B5154A1368154D54152D6A2340ED0727
:10713000ED0F002B04D0002D02D01668A643166078
:107140001668B608B600064316600D48076904269F
:107150003743076101290DD040BF20BF20BF01691F
:10716000B1430161002B04D0002D02D010682043F0
:107170001060F0BD30BFF2E7007000400000014039
:1071800000ED00E0F8B5044600780027534D800676
:1071900071D5524E403EB06BC00004D4B06BA9050F
:1071A0000843B06301274E480168C90511D401683E
:1071B000821511430160FFF7FFFC009005E0FFF727
:1071C000FBFC0099401A642837D845480068C00580
:1071D000F5D532680321090560680A4001409142F3
:1071E00008D08103890F032904D13168890301D5AF
:1071F0000120F8BD2A69032109040A4022D0084071
:1072000090421FD0207880061CD528692A698843BF
:107210000121C9040A432A612A698A432A61286133
:10722000C0050FD5FFF7C8FC009008E0FFF7C4FCCD
:107230000099411A2B48814201D90320F8BD2869E1
:107240008005F3D561688803800F032805D1326873
:107250000005824301400A433260286903226168C5
:107260001204114008432861002F04D0B16B0120A3
:1072700000078143B1632078C00705D0E868A168A2
:10728000800880000843E8602078800705D5E8681A
:107290000C218843E1680843E8602078400706D560
:1072A000E86803218902884321690843E86020785F
:1072B000000706D5E868032109038843616908438C
:1072C000E8602078000606D5E86803218904884331
:1072D000A1690843E8600020F8BD000040100240AA
:1072E0000070004088130000F8B50E46050038D045
:1072F0005E480068C007C00FB04214D25B4C2068E3
:107300004008400030432060FFF756FC074605E088
:10731000FFF752FCC11B564881427AD82068C0074B
:10732000C00FB042F4D12878524C800705D5E068F0
:10733000F0218843A9680843E0602878C00752D04C
:107340006868022806D0032807D0216801280AD0DF
:10735000890504E02168890301E021688901002989
:1073600003DB0120F8BD4907F9E7E16889088900D6
:107370000143E160FFF720FC0746686802280AD055
:10738000032814D001281ED029E0FFF715FCC11BEB
:10739000374881423DD8E0680007800F0228F4D1C9
:1073A00021E0FFF709FCC11B3148814231D8E06878
:1073B0000007800F0328F4D115E0FFF7FDFBC11B88
:1073C0002B48814225D8E0680007800F0128F4D1BE
:1073D00009E0FFF7F1FBC11B2548814219D8E0689D
:1073E0000007800FF5D121480168C907C90FB142D4
:1073F00017D901684908490031430160FFF7DCFBF8
:10740000074608E005E0FFF7D7FBC11B184881429B
:1074100001D90320F8BD15480068C007C00FB0426D
:10742000F1D12878400706D5E06807210902884392
:10743000E9680843E0602878000707D5E06807217D
:10744000C90288432969C9000843E06000F03AF89E
:10745000E168094A0906090F515CC84007490860FC
:1074600007480068FFF7CAFBF8BD00000020024093
:10747000881300000010024066C700088401002045
:107480007C010020044805490068C968044A490590
:10749000490F515CC8407047840100200010024031
:1074A0007FC70008044805490068C968044A890480
:1074B000490F515CC8407047840100200010024011
:1074C0007FC7000870B51A4AD3681A490C201840C3
:1074D0008D0004280CD04E00082810D00C2810D0A5
:1074E00050680004410F0120C003491C884070BD52
:1074F0001068C00601D5084670BD284670BD3046EC
:1075000070BD98020C4C000F205C1B029C0FD368CE
:10751000641CDB0301D5314603E01268D20600D4B7
:10752000294603F01AF922460023FDF7F7FD70BD46
:107530000010024000093D0076C70008FEB50500B6
:107540007ED0FE4CE7680C20E6680740012000046E
:1075500006402878C00747D0082F05D00C2F0AD145
:1075600001200004864206D1206880033CD568686B
:107570000028E5D038E0012069680004814203D189
:1075800021680143216011E0052301221B049204BC
:107590009942216802D111432160F1E781432160C2
:1075A00021680140009120689043206068680028AD
:1075B0000DD0FFF701FB009005E0FFF7FDFA009901
:1075C000401A64287BD820688003F6D50CE0FFF7CA
:1075D000F3FA009005E0FFF7EFFA0099401A6428EB
:1075E000F0D820688003F6D42878800756D5092380
:1075F000E868042F0DD00C2F01D1002E09D00028EF
:107600003CD02168994301432160FFF7D5FA064633
:1076100028E02168490701D5002891D061681F2220
:10762000120291432A691202114361602168994351
:1076300001432160FFF746FFE16809060A0F00E0F9
:107640008BE1BF49895CC840BE490860BE480068FC
:10765000FFF7D4FA002873D120E0FFF7ADFA801BC2
:107660000228AFD820684007F7D560681F210902BB
:10767000884329690902084360600FE020684008D8
:1076800040002060FFF798FA064604E0FFF794FAFE
:10769000801B022896D820684007F7D42878C006B7
:1076A00060D5002F0CD0A86900284AD02068FF219F
:1076B000013108432060FFF77FFA06462EE0C1E063
:1076C0002068800502D5A8690028A6D06068072137
:1076D00049038843296A084360606068297F000283
:1076E000000A090608436060286A410B0120C003B4
:1076F000491C8840E16809060A0F9149895CC84025
:107700009049086090480068FFF778FA002817D180
:1077100028E0FFF751FA801B0228A2D820688005D4
:10772000F7D56068072149038843296A08436060E8
:107730006068297F0002000A09060843606011E0C2
:10774000E2E02168FF20013081432160FFF734FA35
:10775000064604E0FFF730FA801B022872D8206842
:107760008005F7D42878794E000724D56869002869
:10777000306910D0012108433061FFF71DFA0090F5
:1077800005E0FFF719FA0099401A02285AD8306923
:107790008007F6D50FE0400840003061FFF70CFA93
:1077A000009005E0FFF708FA0099401A022849D82E
:1077B00030698007F6D42878400766D5002002900B
:1077C000A06BC00006D4A06B012109070843A06389
:1077D000012002905E480168C90511D40168821534
:1077E00011430160FFF7E8F9009005E0FFF7E4F9C5
:1077F0000099401A642825D855480068C005F5D579
:10780000FF20AA680130824203D13169014331610E
:1078100011E001218902002A07D005231B029A42A8
:1078200003D132690A433261EFE732698243326140
:10783000306988433061A868002810D0FFF7BCF990
:10784000009008E05FE0FFF7B7F901460098091AD9
:107850004048814257D830698005F4D50DE0FFF7E4
:10786000ABF9009006E0FFF7A7F90099411A3948F3
:10787000814248D830698005F5D40298002804D0A8
:10788000A06B012109078843A063686A002866D0BD
:107890000C2F3ED0012636060228206805D0B043C2
:1078A0002060FFF789F905462FE0B0432060FFF71D
:1078B00083F9074604E0FFF77FF9C01B022822D8AE
:1078C00020688001F7D4E96AA86AE2680843296B56
:1078D000FD231B049A4311430843E06020683043B2
:1078E0002060FFF769F9054604E0FFF765F9401BE2
:1078F000022808D820688001F7D530E0FFF75CF94E
:10790000401B022801D90320FEBD20688001F5D468
:1079100025E00128F8D0E06801210904AA6A0140A5
:1079200091421AD10F218904EA6A0140914214D18F
:10793000032189050840296B88420DE000100240B0
:1079400066C70008840100207C010020401002402E
:10795000007000408813000001D00120FEBD00200F
:10796000FEBDF8B504000ED0FF27606A053700257C
:1079700000280AD02561656126464036A562707CE4
:10798000002807D00AE00120F8BD6068B842F3D0B3
:10799000E561F1E73574204600F03EF8022171748C
:1079A0002068026840239A4302602123A26860682D
:1079B0009B021A4038401043E3688A021340184380
:1079C00023690B40217D1843C907C90F0843A169EA
:1079D000931019400843E169382319400843216A8C
:1079E000802319400843A16A930019400843216885
:1079F0000860A0690421000C0840616A1023194046
:107A00000843216848602068C1699143C161656588
:107A1000012070740020F8BD10B586B00446142112
:107A20006846FDF7C4FB10492068884219D10F4809
:107A3000416B821411434163C16A01221143C16247
:107A4000C06A002110400590E020009002200190C3
:107A50000320039002910491052069460007FEF778
:107A6000DBFF06B010BD00000030014000100240F6
:107A7000094910B5401E884201D9012010BD074CAC
:107A800060610321081F02F0A3FE0020A06107200F
:107A90002061002010BD0000FFFFFF0000E000E0BB
:107AA000F0B502462032137E012B1ED0012515763B
:107AB0000223537606687468B3687027BC430F6866
:107AC000274377600068AC07A04205D0084CA0426D
:107AD00002D0084CA04204D180244968A343194332
:107AE0008160557600201076F0BD0220F0BD0000C8
:107AF000000801400014014070B5050005D02C4677
:107B00002034607E002802D006E0012070BD0020F5
:107B10002076284600F010F802206076291D28689B
:107B200002F08CF80120A077A076E07620776077CD
:107B30006076002070BD000000680121890788423E
:107B400004D10348816B0122114381637047000017
:107B500000100240F8B5054604462035287E01286D
:107B600017D001262E760220687622689068772743
:107B7000FF23B8431B02984390600A68502A31D013
:107B80000EDC202A4BD006DC002A48D0102A3AD13D
:107B900045E00220F8BD302A41D0402A33D136E0FA
:107BA000602A27D0702A12D001200003121A2AD08E
:107BB000824228D1CB684A688968206802F077F849
:107BC0002068816801229203114381601BE0CB6829
:107BD0004A688968206802F06AF821688868384332
:107BE000886010E0CA684968206802F0DAF850211D
:107BF000206806E0CA684968206802F0E3F860215E
:107C0000206802F05FF86E7600202876F8BDCA681A
:107C10004968206802F0C5F840212068F1E7114664
:107C20002068EEE710B586B0044614216846FDF7DB
:107C3000BEFA012120688907884212D10A49CA6A1E
:107C400002200243CA62C96A0190014005914102C3
:107C50000091002102910391049069460348FEF7C8
:107C6000DBFE06B010BD0000001002400004005012
:107C7000F8B5064604462036307E0D4601280BD066
:107C8000012008273076002A08D0042A16D0082AB6
:107C90002AD00C2A4DD137E00220F8BD206802F02E
:107CA00019F820688169394381612068816904225B
:107CB0009143816120688169EA6812E0206802F0DE
:107CC00021F8206881690122D20211438161206874
:107CD0008269012189028A43826120688169EA6898
:107CE00012021143816124E0206802F024F8206828
:107CF000C1693943C1612068C16904229143C161EE
:107D00002068C169EA6812E0206802F02FF8206854
:107D1000C1690122D2021143C1612068C2690121F7
:107D200089028A43C2612068C169EA68120211436C
:107D3000C16100203076F8BD70B5050005D02C4635
:107D40002034607E002802D006E0012070BD0020B3
:107D50002076284600F00FF802206076291D28685A
:107D600001F06CFF0120A077A076E07620776077A5
:107D70006076002070BD704770B505462C46022025
:107D80002034002908D004290BD008290ED0627FA6
:107D9000012A10D0012070BDA27E012AFAD1A0765E
:107DA0000AE0E27E012AF5D1E07605E0227F012A91
:107DB000F0D1207700E060770122286801F06AFFA7
:107DC0000122286892070121904205D0074A90427B
:107DD00002D0074A904204D182685207520F062A05
:107DE00002D002680A430260002070BD0008014012
:107DF0000014014070B504460D460068002201F0F1
:107E000049FF2068016A0C4A114203D10168490800
:107E10004900016001202034002D06D0042D06D039
:107E2000082D06D06077002070BDA076FBE7E076D5
:107E3000F9E72077F7E7000011110000704770475D
:107E400070470000F8B502680446D069116896686A
:107E5000814B05461D402023002D6CD0F7077F4D38
:107E6000FF0FBC460D402F4379D02546C70780350C
:107E7000002F06D0CF0504D5012717622A683A43A0
:107E80002A60820708D5F20706D0276802223A62E4
:107E90002A6804273A432A60420708D5F20706D029
:107EA0002668042232622A68022632432A600207C8
:107EB0000AD50A461A406646324305D0266808228B
:107EC00032622E6816432E60020508D54A0106D597
:107ED00001222668D20232622A681A432A602A687E
:107EE000002A30D0800606D5880604D5616E0029A8
:107EF00001D020468847286821688968490602D44D
:107F00002821084225D0204602F073F920688168B4
:107F1000490619D5826840218A438260206F002873
:107F200012D04F498163206FFEF7DCFB00280AD096
:107F3000206F816B06E0850611D58D060FD5616E29
:107F400077E020468847F8BD2046FFF779FFF8BD67
:107F500005E02046FFF774FF00202860F7E7256E54
:107F6000012D56D1C50654D5CD0652D51026166220
:107F70002068816825464906403500292ADA226FA3
:107F8000116849680904090CE1D02F8B8F42DED9B2
:107F9000698311680968890617D401683201914321
:107FA0000160206881684908490081602068816813
:107FB000402291438160E3670020206620680168C9
:107FC000B1430160206FFEF76BFB288B698B401A71
:107FD00081B21AE0298B6A8B891A6A8B89B2002ACE
:107FE000B5D00029B3D00268FF252135AA4302602D
:107FF00020688268520852008260E3670020206691
:10800000606620680268B24302602046FFF716FFF0
:108010009DE7C50208D5750206D50120000510624E
:108020002046FFF70CFF92E7050605D50D0603D5A0
:10803000A16E002985D18AE7400688D5480686D5F5
:10804000116820464024A1431160836700218166A6
:1080500000F043F97BE700000F0800002001000456
:1080600019A1000810B5040003D0A06F002802D0A9
:1080700007E0012010BD002174200155204600F0CA
:1080800027F82420A067206801684908490001609A
:10809000204602F001F90128ECD0606A002802D0E5
:1080A000204601F023FF206841680922D202914353
:1080B0004160206881682A229143816020680168BC
:1080C000012211430160204601F076FF10BD00003F
:1080D000F0B587B0064614216846FDF768F82C49CC
:1080E0003068884251D12B48416B012292031143E1
:1080F0004163C16A01221143C162C06A0025104078
:1081000005900320400200900220032701A9A1C18D
:1081100004200490052069460007FEF77DFC1F4CF3
:108120001D48A560E56081C48027E560A760202028
:10813000256160610002A0611848083CFEF74CFB15
:10814000002801D0FDF7FEFD3467A662144C1248EA
:108150002146143820600320606010200831A1C13E
:108160006561A561E56120462562FEF735FB0028C3
:1081700001D0FDF7E7FDF466002201211B20A66275
:10818000FEF7A2FF1B20FEF793FF07B0F0BD000033
:10819000003801400010024030000240501700201B
:1081A0009817002070B5C36F202B27D100290BD062
:1081B000002A09D0012483682403A34206D103695D
:1081C000002B03D1CB0701D0012070BD03466033E3
:1081D0001C7D012C12D001241C7500230366084C61
:1081E0000368A34207D05C68240204D51C680125FB
:1081F000AD062C431C6002F04FF970BD022070BD2B
:108200000048004070477047FFB50446806F83B058
:1082100017460D4620285ED1002D0AD0002F08D029
:10822000A168C001814207D12069002804D1E80774
:1082300002D0012007B0F0BD204660300090007DE4
:10824000012848D0009801210175002080210851A3
:108250002120A067FEF7B0FC264640360190378209
:1082600077820120A1680003814202D120690028A1
:1082700005D02F46002500990020087511E0002741
:10828000F9E700228021204602F04CF9002815D1A0
:10829000002F15D02168387888627F1C708A401EB4
:1082A0007082708A019B002806980090E9D1002214
:1082B0004021204602F036F9002808D00320B9E713
:1082C00028882168C005C00D8862AD1CE6E7202023
:1082D000A0670020AEE70220ACE77047034D044CD6
:1082E00004A002F019FAE560FAE700000400FA05BC
:1082F00000ED00E0486172644661756C745F48612E
:108300006E646C65722E0D0A0000000000B585B029
:1083100014216846FCF74BFF03480221418300F01B
:10832000EFFB05B000BD00003C01002010B50524A6
:108330002407002204212046FEF737FC00220821F2
:108340002046FEF732FC0A2002F04BFC01220421F9
:108350002046FEF72AFC0A2002F043FC00220421FA
:108360002046FEF722FC10BD10B50524240700228C
:1083700004212046FEF719FC012208212046FEF7C1
:1083800014FC0A2002F02DFC012204212046FEF7F5
:108390000CFC0A2002F025FC002204212046FEF7F6
:1083A00004FC10BDF8B5002405260746254636070F
:1083B000002204213046FEF7F8FB0A2002F011FCEF
:1083C000012204213046FEF7F0FB6006040E08216E
:1083D0003046FEF7DDFB002801D0641CE4B2052026
:1083E00002F0FFFB6D1CEDB2082DE1D3002F03D08E
:1083F000FFF79CFF2046F8BDFFF7B6FFFAE770B520
:10840000052605463607002204213046FEF7CDFB3F
:108410000024E80901D0012200E0002208213046B2
:10842000FEF7C3FB6806050E0A2002F0DAFB012204
:1084300004213046FEF7B9FB0A2002F0D2FB0022ED
:1084400004213046FEF7B1FB0A2002F0CAFB641C8F
:10845000E4B2082CDDD370BD10B505242407012239
:1084600008212046FEF7A1FB012204212046FEF749
:108470009CFB002208212046FEF797FB0A2002F011
:10848000B0FB002204212046FEF78FFB10BD10B583
:1084900005242407002204212046FEF786FB002243
:1084A00008212046FEF781FB0A2002F09AFB0122F8
:1084B00004212046FEF779FB012208212046FEF721
:1084C00074FB0A2002F08DFB10BD70B505252D0749
:1084D0000024012208212846FEF767FB062002F04F
:1084E00080FB012204212846FEF75FFB062002F0F4
:1084F00078FB07E0641CE4B2FA2C03D9FFF7C7FF4E
:10850000012070BD08212846FEF742FB0028F1D16A
:10851000002204212846FEF748FB002070BD000021
:10852000F8B501F07BFD01F0ABFD5B480068C06968
:10853000FDF7F8FC594C5A49A082898F594E002505
:10854000002931D0A26A730357499A4202DB022202
:108550000A7000E00D700A7801218902002A05D016
:10856000012A0ED0022A10D0032A1DD1608B0128C7
:108570002ED0022818D1484808214038FFF73AFC8D
:1085800012E0FF22F5329042F0D2608B01281DD01C
:10859000022804D008E03046FEF707FB04E03E481E
:1085A00008214038FFF7E8FBFDF7C6FD20700121E8
:1085B000C9023046FEF7ECFA0127FF0300282DD050
:1085C0003A480560A079002804D007E00022E2E7DD
:1085D0000122E0E70120A07102F006F88021304678
:1085E000FEF7D6FA002806D0002208213046FEF712
:1085F000DCFA012205E0012208213046FEF7D5FA17
:108600000022052039460007FEF7CFFA244C284EF9
:108610004034A08C274F012803D01CE0A571002214
:10862000EAE725486946088072B680212348FDF7AD
:10863000A1FB002804D0022269462048FDF73EFC39
:1086400062B61FA002F068F8A58403F09FFF6420C3
:1086500002F0C0FAFE60608C012808D110486584E1
:10866000058003F093FF642002F0B4FAFE60208CD2
:10867000012806D1258403F089FF642002F0AAFABC
:10868000FE600748124A0188914202D1C088002842
:1086900000D1FE60F8BD0000CC1600203C01002097
:1086A000E80D00200004005081000020740100202B
:1086B0000400FA0500ED00E0AAAA0000384A00080C
:1086C000BDF8C8EBC9FDBCB6C4A3CABD0D0A000005
:1086D000AA55000008B55721202000F06AF80321B0
:1086E000212000F066F84021222000F062F80821E5
:1086F000232000F05EF8AA21302000F05AF8084844
:1087000001210187322000F054F80221332000F0CB
:1087100050F8684600F006F80A2002F062FA08BD38
:10872000E80D002010B501460F2000F021F80028C8
:1087300000D0012010BD10B50446FFF78DFE322099
:10874000FFF75DFEFFF7C1FEE0B2FFF758FEFFF74F
:10875000BCFEFFF781FE3320FFF751FEFFF7B5FEA9
:108760000020FFF71FFE0446FFF791FE204610BDD4
:1087700010B50C46FFF7DFFF2070012010BD70B56B
:108780000D460446FFF768FE3220FFF738FEFFF77C
:108790009CFEE0B2FFF733FEFFF797FE2846FFF797
:1087A0002EFEFFF792FEFFF772FE0A2002F019FA82
:1087B00070BD10B5FFF7E3FF012010BD10B50248F2
:1087C000FEF735FB10BD000004160020FEB5044680
:1087D000002772B6334A01688B1804D13248C76843
:1087E00003208004074088680190C86800904869A9
:1087F0008E69002B08D12C4940398B6ACD042B435C
:108800008B628B6AAB438B62014631433CD0254976
:108810002368CB4205D12449CA6803239B049A43A9
:10882000CA6025462035002810D021680A69012336
:108830001A430A61216848610821204600F036F891
:10884000032800D1A873216808204860002E10D0AA
:1088500020680169012211430161206886611021AD
:10886000204600F023F8032800D1A87321681020C7
:1088700048600C482168C14206D10B48C1680322F8
:10888000920491433943C160206801694908490055
:10889000016121680198886021680098C86062B60B
:1088A000FEBD00000084FFBF4010024070B50646C8
:1088B0000B480D46002409490068FCF719FC7D218E
:1088C000C90048433168401E00D103240B682A4682
:1088D0009A4301D00028F6D1204670BD204E0000FA
:1088E000840100201CB5002116480091144A019112
:1088F0000260C16312054260816007228263012227
:1089000002610246C16020321170FF235170C233F0
:108910004362816211730163816104224163426198
:10892000C161FDF723FD084800908013019069465E
:108930000448FDF7CBFC00210248FDF771FC1CBD8B
:1089400000240140A81500200200000408B50848D2
:10895000016B012211430163006B01211040009063
:1089600000220A20FEF7B0FB0A20FEF7A1FB08BD9B
:1089700000100240F0B587B014216846FCF717FCE0
:108980004748C26A04210A43C262C26A0A40059289
:10899000C16A80263143C162C16A31400591C16A12
:1089A00001242143C162C16A21400591C16A0225A7
:1089B0002943C162C06A22462840059005201C2137
:1089C0000007FEF7F2F8012236493748FEF7EDF8C6
:1089D000002236493448FEF7E8F8912105200022AC
:1089E00009020007FEF7E1F8314801900027052051
:1089F0006946029700940007FEF70EF80C200090DD
:108A0000112001900320039005200297694600077A
:108A1000FEF702F810206A46039591C205206946C8
:108A20000007FDF7F9FF11200190029769460397AF
:108A300000941D48FDF7F0FF1E480190694600951F
:108A400002941948FDF7E8FFE0020090694601979B
:108A500002951548FDF7E0FF1748694691C1694640
:108A600011480397FDF7D8FF91200002694691C194
:108A70000520694600070397FDF7CEFF69460A48BF
:108A8000019700960294FDF7C7FF002201210520FF
:108A9000FEF71AFB0520FEF70BFB07B0F0BD000048
:108AA00000100240010200000004005008300000E5
:108AB00000001110000021100832000010B50F4C0A
:108AC0000D482060FF20053060600020A060E0605D
:108AD00020616061E0610121206249026062A16160
:108AE000A0620720E0622046FEF73BFF2068016895
:108AF00040221143016010BD0030014034160020B7
:108B000010B58AB000240494059406940794089440
:108B10000121184809940094019402948907039450
:108B20000160092184604160046113494461C160AE
:108B3000FEF7E2FF01200003049004A90D48FFF7AF
:108B400009F80C48FFF7F8F8089408A909480994AF
:108B5000FEF7A6FF602000900848019002940822CA
:108B6000694603940348FFF783F80248FFF75AF871
:108B70000AB010BD8C1600209304000057020000BC
:108B800000B585B014216846FCF711FB0E480D496D
:108B90000160E1214902416000218160C160016101
:108BA00081610C22C1614261016230214162012177
:108BB000090381634900C163FFF754FA01F00EFD18
:108BC00005B000BD00380140CC1600207047000001
:108BD000F0B589B00A2002F04FFD7D20400102F07F
:108BE00065FDF84C0025A570F748E065A07B0C28D2
:108BF00001D30B20A07360790A2801D90A20607183
:108C0000F248E570F24E00783071F249A0790978A7
:108C100040000843E17C89000843F071A06BF070CC
:108C2000010A3172401CA0636079B0744200304682
:108C3000E9491330FCF7A2FA6079E7498200400065
:108C4000801960311330121DFCF798FA6079062103
:108C5000420048438019E1491730921CFCF78EFA14
:108C60002A20205E002803D0DD49098A0818608583
:108C70006079D449C000223182190B7A53764B7A3D
:108C8000937606227272D74A1D301278B272228C05
:108C90003273CF4A0B78133A137549785175002215
:108CA000CB4902F0D3FD60790021C0001D3002F0F5
:108CB000DFFDCD48FEF796F90127A084BF0309E048
:108CC000C948FEF78FF980B2A084618EFF392D3933
:108CD000884206DB618E80B28842F1D3C91988428E
:108CE000EED8022002F018FDB9480126C571E573DF
:108CF000E57266732573BC48FEF774F9E084074695
:108D0000E5706079FCF7DCFCB84AB94BFCF7BCFBBA
:108D100001F0FCFE0022B74BFCF704FBFCF716FD4C
:108D20000006C00CC01980B2F1032085884201D32F
:108D3000401A2085B048A0642079401C2071AA48C0
:108D4000FEF750F9A084A4489E4F6438403706903F
:108D5000B4E1A548FEF746F9A0840BE0A248FEF76F
:108D600041F980B2A084218D884203D3A34A891897
:108D7000884207D300210F2002F0FEFBA049E063E8
:108D80000842EBD0E06B411C20D040047ED581220C
:108D9000D20100210F2002F02EFD7D20400102F0C3
:108DA00085FC002002F037FC0021102002F0E4FBDB
:108DB00041068948490E00227C38A16502F012FC68
:108DC00085487C38417A0729C2D101E001F022FDB3
:108DD00002228C49401DFCF7F5F90028B8D102F0B9
:108DE00098FDE167A06702F081FD764B803303C3F5
:108DF000E0787949401CE07083390B7A684603704B
:108E0000497A417000880390618C88427ED1704914
:108E10007D488C31C98E01806D496A488C31098F3B
:108E2000C1837148FEF7DEF8A08402F0B7FA654806
:108E3000FF2280300168406852040023891858419D
:108E40000206080A10434108490000900A0E080271
:108E50005C498031CA6088605D48E36F0A30A26F68
:108E600002F02CFD607981005948081855491630E8
:108E700080310CC902F022FD52488030C3688268FC
:108E80005348123002F01AFD082100E009E1504871
:108E90004172B430C07C0009A07414D04E48022244
:108EA00058497738FCF78EF900280CD14848E6730A
:108EB000C671A06D48491638C2B26639C81D227401
:108EC000FB30FCF75BF960790022800040491C30E0
:108ED00002F0BCFC6079002180001C3002F0C8FC6C
:108EE000009802F0C2FB012002F016FC6072022121
:108EF0004648FDF74DFE00281DD00020354908707A
:108F000033498C31488E0490B88000E082E0888E2E
:108F1000F8808446606CFF310531A0640860DC395C
:108F2000E064C97C0907090F032900D06174A16DB1
:108F30001C2902D015E00120E0E72549214A8C31A7
:108F4000C98F9185069B254A1B881380884207DDBF
:108F5000002805DD002903D0607D401C607500E01D
:108F600065752571E67204983881604678812673AC
:108F7000E08B2749FF30C33080B2E08388420CD9B0
:108F800049424018E08320487D220188D200491CD4
:108F900089B20180914200D305801B4801887D2061
:108FA000C0004143E08B0818206500F06DFD607A39
:108FB000002805D100210F2002F0DEFA0006F9D5C5
:108FC00085E00000700000203F420F003C010020BF
:108FD0005C120020700100208C130020C8140020B7
:108FE000280E00204C01002004160020B81E85EB3E
:108FF00051B8CE3F00000840A0860100983A00001A
:1090000000D02724600100206C01002000040050E3
:10901000E7030000FCF76EFF674A0321115467491C
:109020004A8EBA80898EF980A26D1C2A06D1624BC5
:109030004200AC33D318069A12885A8080005E4AE8
:109040005E4B603A02905C4982189B8F13803039E6
:109050004118626C4A6059498C3940185849163099
:109060000CC902F02BFCE16D606C884208DA524AB0
:109070000299603A5158012902D1E065039905919E
:109080004D49029A60398A58824217DD012A15DD5E
:109090002146002812DD0398488402200870A5723A
:1090A0000CE0484A00210F2002F0A5FB6079E1782E
:1090B000401C814202D0002002F0ADFAA18C208D2C
:1090C000814200D245E6404A80188142FAD8E07ACF
:1090D000012801D00220E07202F060F9394A002133
:1090E0000F2002F088FB2179002914D0374800882E
:1090F000820082188A4200D22570002000F0E0F839
:10910000E07B002836D02C490C310B7848788A78DF
:10911000022B17D02EE0A16CE06D323988420FDAB5
:10912000E1792A4A491CC9B2E171128820465200ED
:109130008A42E5D20599418402210170A572DFE7D8
:10914000E571DDE710280CD0C82813D2204BC91CCC
:109150001818FCF713F803F019FA642001F03AFD2F
:1091600034E61C4D28684000000E03D1C878FCF797
:109170008CFA286000202278A37A65790FE00E4EE1
:109180004100903E775A1836765AB74205D00B4FB9
:109190000222002301268C377E52401CC0B2A84216
:1091A000EDD32270074AA372803200210F2002F013
:1091B00022FB09B0F0BD00001C140020E8120020C2
:1091C000F000002000D02724983A00004C01002035
:1091D000E80D002064010020F8B52E4C0546A06E75
:1091E0002D4A281A411EE066914215D2EB218900D2
:1091F000081AFCF751FA294A294BFCF745F90646AB
:109200002E200F46205EFCF747FA32463B46FCF71D
:1092100089F8FCF777FAE0850020A0751D4818232F
:10922000C35E028C1F48008884461F4806881DE0E4
:109230006046484380181D4F80B2388030277843FD
:109240006427643078431A4F2066C01985420BD2D8
:10925000C8B218492E220880206EA25E411BC91890
:1092600089186166A066F8BD491CA175A17DB1424F
:10927000DED33020424310486421101848430F4980
:109280004118A16620662E21401B615EC01840185F
:109290006066F8BD70000020CF0700009A99999988
:1092A0009999B93F5A0100204C0100206E0100201D
:1092B00078ECFFFF5801002074270000C0BDF0FFCC
:1092C000F1B5284882B00188491C8FB20780264832
:1092D000068826483146FBF70BFF254CA18E451822
:1092E000B74205D31F48002101802248281811E009
:1092F0000298FCF7E5F9204A204BFCF7C5F8064632
:109300000F462846FCF7DCF932463B46FCF70AF8E4
:10931000FCF71CFA2086012580B2ED03A84201D398
:10932000401B2086608BFCF7CBF9154A154BFCF7E8
:1093300013F90746208E0E460090FCF7C1F93A4615
:109340003346FBF7EFFFFCF701FA80B26086A842D4
:1093500001D3401B60860C49009809684861009859
:10936000A086FEBD580100204C010020E17A0000DB
:1093700070000020240500001904560E2D624040A4
:10938000F853E3A59B843E4004160020704700007C
:10939000F0B589B0002004900A2002F06DF97D201C
:1093A000400102F083F9B34800218170826BB34C15
:1093B000521C8263B04A438D128A2546D2184285D8
:1093C0000175214613310791223047310290313522
:1093D00020461338AA4F03910590A64E0F21A948A5
:1093E000717100782071A84AB0791278400010435A
:1093F000F27C92001043E071308FE070000A20721E
:10940000A17431461E229C310798FBF7B7FE40221B
:1094100028469E49FBF7B2FE029903980A7AC27465
:10942000497A01750920607299480078A072308CE1
:109430002073307D410030469C30091805980A7829
:10944000027549784175762000228C4902F0FEF9B8
:1094500070790621484300211C3002F009FA0220ED
:1094600002F05AF900210F2002F086F83842F0632A
:10947000F8D0F06B411C18D040047DD58122D20178
:1094800000210F2002F0B7F90021102002F074F83B
:1094900041067A48490E0022B43002F0A3F877481A
:1094A000B430417A022902D0BDE001F0B3F90222C2
:1094B0007849401DFBF786FE0028F5D16D48022251
:1094C000007D41006B489C3009186C48B530FBF7B3
:1094D00079FE0028E8D102F01CFA664AD16790674D
:1094E00002F004FA634A803203C2049800282CD1A7
:1094F000012004906148684E8C30C08E5F493080F6
:109500005C488C31098FC1836448FDF76BFD594974
:10951000634A8884C88BFF30C33080B2C8839042CE
:109520000CD952428018C88330885D4A401C80B2F2
:109530000B323080904201D30020308030887D2271
:10954000D2005043CA8B801808654C4869468C305D
:10955000428E0A80808E488048490422B531C81F57
:10956000FF38FBF70BFE4348484A007D0099800016
:1095700011504049803100E076E003C9FF235B04CD
:109580000022C01851410906060A0E43304602F077
:109590006CF8710849000A0E08023649002680312D
:1095A000CA6088603348C36F826F3448483802F01D
:1095B00085F9304880300CC83048443802F07EF9D4
:1095C0002C488030C36882682C48403802F076F915
:1095D0002A49002252393C2002F038F900213C206F
:1095E00002F046F9012002F097F822494872084635
:1095F0008078401C887001210520C9030007FCF712
:109600008DFC1C48407A002805D100210F2001F074
:10961000B3FF0006F9D5802200210F2002F0EBF8FD
:109620001448467002E01349012048701148017D3A
:10963000491CC9B201750F2900D2CEE60498002852
:1096400010D10C481749028C002A02D00B889A428C
:1096500001D9098801841449008C0988401E4843B7
:109660001249088009B0F0BD114A00210F2002F014
:10967000C2F8D8E770000020280E00205C120020FD
:1096800000D027243C010020700100207814002025
:109690004C010020600100206C0100200416002015
:1096A000E70300004801002046010020440100209B
:1096B00000902724F8B531492F48086002F00AFAD3
:1096C0002F4800F0A1F92F4CE0822D48801C00F0BB
:1096D0009BF920832A48001D00F096F960832B48EF
:1096E00029494180014640310979294F0906090E6F
:1096F000617006D1C7800121C1870A2141870021FD
:109700008187244AC18E1170C18F2171818F61714F
:10971000817AA1708588052165626181C68830469D
:10972000FBF7E6FCA08101462846FBF7E1FC880038
:10973000081885B2164825816843FBF7C1FF164A11
:10974000164BFBF709FFFCF701F8E0816582314613
:109750003846FBF7CDFC20820146C820FBF7C8FC49
:10976000E0830120A083FCF7DDFBA082E2890C49A5
:109770000C48FDF73BFCF8BD09A600086800002076
:10978000004F00083C01002029020000E80D0020E5
:10979000E803000018000020F853E3A59B843E4036
:1097A000FF7F000004160020F8B5744C00202071E3
:1097B000734D01202880734EC8203080207A401CD1
:1097C0002072C00706D0208C411E2184022801D2BD
:1097D000C82020840120FFF773FD0A2001F04CFF10
:1097E0007D20400101F062FF02216748FDF7D0F9BA
:1097F00000283FD00020654980000978654F490066
:109800000843634909780843B872102078726248A7
:10981000C1887D20C000FBF76BFC78735F485E4910
:109820000078B87338460B308A780270C978417076
:109830005949421C20310B7ED370497E1171564923
:10984000D01C22310B7E5371497E917152494031B7
:109850000A7C0271497C417100223946172001F0CF
:10986000F5FF0021172002F003F8022001F054FF59
:109870004B4F03E00120BEE7FEF752FE00210F2010
:1098800001F07AFE3842E063F6D0E06B411C73D001
:1098900040046FD58122D20100210F2001F0ABFFDF
:1098A0000021102001F068FE41063A48490E0022CE
:1098B000B430A16501F096FE364FB437787A11289E
:1098C00058D102223749781DFBF77CFC002851D182
:1098D000F81F027A69460A70407A4870B97A29807E
:1098E000C820FBF705FC3080387B208438462E4D9D
:1098F0002838C08E2880394620482839098FC183EE
:109900002A48FDF76FFBA084E08B2949FF30C33064
:1099100080B2E08388420CD949424018E08328880D
:109920002349401C80B20B312880884201D300209B
:10993000288028887D21C9004843E18B4018206594
:1099400000F0A2F86846008860841249B87CC731EC
:109950006071420008460D466930FBF70FFC6079E4
:10996000294642001348FBF709FC208CFF2801D050
:1099700003202070F8BDFFE700F04CFF70000020CE
:109980004C0100205A01002000040050400100203A
:10999000410100205C120020E80D0020180000208A
:1099A00000D02724600100206C0100200416002054
:1099B000E7030000A413002070B586B014216846A8
:1099C000FBF7F5FB01250F4EED030022294630463B
:1099D000FDF7EBF801200024019002946946009500
:1099E00003943046FDF718F803200190029469466D
:1099F000009503943046FDF70FF8022001F0EAF8D5
:109A000006B070BD00040050008870477047000029
:109A1000F8B5044600206A461080194D55222A7078
:109A2000AA226A700322AA70661DEE702A716971FB
:109A3000144A49008918AC712246E81DFBF79EFBC9
:109A4000002007E029186A468978128889186A4632
:109A50001180401CB042F5DB611DA81CFCF7C2F868
:109A600001466846018029190078C8716846407827
:109A7000087221460931024800F0DCFBF8BD000005
:109A800042150020E80D0020FEB5FFF7A5FB254894
:109A9000FDF7A8FA244C86B2A68460790A21081A38
:109AA000C000FBF7F9FD07460191606EFBF708FE69
:109AB0001E4A1F4BFBF750FD00900D463046FBF74A
:109AC000FFFD2B46009AFBF72DFC3A46019BFBF766
:109AD00029FCFBF73BFE85B22586608BFBF7F0FD8A
:109AE000124A134BFBF738FD06460F462846FBF794
:109AF000E7FD32463B46FBF715FCFBF727FE81B23C
:109B00000120C0036186814201D3091A6186854222
:109B100001D3281A20860349208E09684861A0864F
:109B2000FEBD00000416002070000020F853E3A5DD
:109B30009B843E40034A1168382389B2994301430C
:109B4000116070470030014010B5FDF73BF810BDC3
:109B500010B59AB034216846FBF729FB14210DA8F3
:109B6000FBF725FB1C2112A8FBF721FB1B48016812
:109B70000324E402A143C21489180160FDF7B0FA7E
:109B800017480169A143016106200090FF200130C0
:109B900002900120039010200490022009904004BC
:109BA0000B90000100240C900A946846FDF7C6FC57
:109BB0000F200D9003200E900F941094012111940A
:109BC0000DA8FDF791FB81201290032080041890CE
:109BD000149412A8FDF7D6FA1AB010BD0070004018
:109BE0004010024010480168821511430160C168AD
:109BF0000E4A1140C16001680D4A11400160816840
:109C00004908490081600168012292049143016082
:109C1000C168FD2212049143C1600021016106491F
:109C20000448886070470000001002400C40FF8824
:109C3000F6FFF6FE0050000800ED00E070B5026887
:109C400001239B07114C124D984203D0A04201D032
:109C5000A84203D17026B2434E683243984203D0E3
:109C6000A04201D0A84204D103231B029A43CB682F
:109C70001A4380239A430B691A4302608A68C262BE
:109C8000096881620121416170BD00000008014046
:109C90000014014010B5CB06DB0E0121046A994087
:109CA0008C430462016A9A401143016210BD30B5D1
:109CB0008468FF252D021B021343AC430B4323434F
:109CC000836030BD826870239A430A4307210A43A8
:109CD0008260704730B5026A520852000262026A1E
:109CE000456883697024A3439C080B68A400234340
:109CF0000224A2438C684560144383614968416330
:109D0000046230BD30B5026A10239A430262036ACE
:109D10004568826973242402A2430C682402144318
:109D2000202293438A68456012011A43846149687E
:109D30008163026230BD30B5026AFF2301339A436A
:109D40000262026A4568C3697024A3439C080B68D9
:109D5000A400234301246402A2438C6845602402CA
:109D60001443C3614968C163046230BD30B5026AFF
:109D700001231B039A430262036A4568C269732484
:109D80002402A2430C682402144301225203934389
:109D90008A68456012031A43C4614968016402621B
:109DA00030BD30B5036A046A6408640004628469E3
:109DB000F025AC43120122430A24A3430B438261E2
:109DC000036230BD30B5036A1024A3430362846983
:109DD000036A0F252D031203AC432243A024A3439F
:109DE000090119438261016230BD0000F8B51024F9
:109DF00005252D07AC62AF20800000F0F2FEAC61BB
:109E000001F0CEFB2F4C304F304E20670EE001F0BA
:109E1000C7FB2067FEF784FB206C411C21641428DB
:109E200004D92BA000F078FC2D48C760206FB04209
:109E3000EDD10026266420780127FF03030000F0FF
:109E4000A4FC05040C192D303200012239462846A5
:109E5000FCF7ABFEFFF7A8FC06E0012239462846D6
:109E6000FCF7A3FEFFF794FA002239462846FCF7D8
:109E70009CFE18E0A07A0122401CA07239462846B8
:109E8000FCF793FEFCF76AF8002239462846FCF7F7
:109E90008CFEA07A052806D9267004E0FEF798FE0D
:109EA00001E0FFF775FA02210E48FCF771FE002869
:109EB00005D000200C49087001F058FAF8BD0120C7
:109EC000F8E70000700000200400FA053001CADE47
:109ED0004457204944204552524F522E0D0A00004B
:109EE00000ED00E0000400507001002010B5818CEE
:109EF000C90707D001684A6801235B049A43836A53
:109F00001A434A60818C890707D501684A68012392
:109F10001B049A43C36A1A434A60818C490707D5D8
:109F200001684A6801239B049A43036B1A434A6001
:109F3000818C090707D501684A680123DB039A432E
:109F4000436B1A434A60818CC90607D50268916841
:109F500001231B039943836B19439160818C89060C
:109F600007D501688A6801235B039A43C36B1A43D0
:109F70008A60818C490612D503685A680121090557
:109F8000046C8A4322435A60026C8A4207D10268F9
:109F9000516803235B059943436C19435160818CDD
:109FA000090607D501684A680123DB04806C9A43DF
:109FB00002434A6010BD0000F8B504460026803018
:109FC0000660FCF7F9FD054620680068124F00079F
:109FD00009D501212B46002249052046009700F0B3
:109FE000A1FA00280DD12068006840070BD5012197
:109FF0002B46002289052046009700F093FA00289E
:10A0000001D00320F8BD2020A067E06726666034F9
:10A0100026750020F8BD0000FFFFFF01F8B5154CC4
:10A02000C826E078002823D16079002820D10120BB
:10A030006071114D686B0027002818D0686BC8212B
:10A04000081A0FE00D48E168405C61698847E068E4
:10A05000401CE060E068C82800DBE760696BC8204E
:10A06000401A761EE168814201D0002EEADC677159
:10A07000F8BD00005400002000000240200D002028
:10A0800070B5224CE07800283FD1207900283CD1DF
:10A09000012020711E4EF16900250906002933DADE
:10A0A0002156625791420AD1F06940062CD5A07919
:10A0B000002829D0A5712089401C208124E0A179A5
:10A0C000002903D1A0710A2000F08BFD002020564A
:10A0D000CC2148430F494218206912181279B26204
:10A0E000401C00222061A256CC235A438958814249
:10A0F0000ADC25612078401C207020780E2800D1D1
:10A100002570A078401CA070257170BD54000020FF
:10A1100000380140F801002010B5806A0022014695
:10A1200040314A834A82FDF78BFE10BD70B5846AC8
:10A13000A06FE56F2168896800260906002906DA04
:10A14000212804D152200653204600F06BF82068E5
:10A150008068400606D5222D04D15A200653204699
:10A1600000F047F82046803001681022114301605A
:10A170002046FDF765FE70BD10B501460968806A8E
:10A18000096889061CD400225A210A5201680A680B
:10A19000FF2301339A430A6001688A68520852001B
:10A1A0008A6001688A6840239A438A602021C167D7
:10A1B000016E012904D101680A6810239A430A60DC
:10A1C000016E012902D0FEF71DF810BD5821095A71
:10A1D000FDF734FE10BD10B5806A016E012902D072
:10A1E000FEF711F810BD5821095A4908FDF726FE5F
:10A1F00010BD01680A68FF2321339A430A60016891
:10A200008A68520852008A60016E012904D10168EF
:10A210000A6810239A430A602021C1670021016661
:10A220004166704701680A68C0239A430A6020218A
:10A230008167704770B5164CE278002A0CD12279FC
:10A24000002A09D10122E2700025C82903DC02227C
:10A25000A256002A01DCE57070BD0123E356CC2232
:10A2600053430C4AD1500123E356CC2673439B1829
:10A270000A460146181DFAF781FF6078401C60709D
:10A2800060780E2800D16570A078401EA070E2E7CB
:10A2900054000020F8010020F8B5044601688068E9
:10A2A0002369E66918436369002533431843724AFA
:10A2B0000B68724E334003430B60216848680323E8
:10A2C0001B039843E368184348602168A0699142E2
:10A2D00001D0236A18438B680B263602B34303432D
:10A2E0008B606749236867488B420CD1C068800740
:10A2F000800F06D0012839D0022835D0032821D17B
:10A300001EE001271FE060498B420AD1C0680C2182
:10A31000084027D0042829D0082825D00C2811D19E
:10A320000EE093420ED1C16803208002014019D093
:10A3300001208002091A19D0091A15D0814201D1D1
:10A34000082700E010274F495048403986009342C3
:10A3500032D1002F0CD0022F0DD0042F10D0082F97
:10A360007FD126E00027EEE70227ECE70427EAE7A3
:10A37000FDF788F806E00968C90605D4304603E011
:10A38000FDF7A0F8002872D0626851005118814290
:10A3900067D81103814264D3010E060250080023DE
:10A3A00030185941FAF7BAFE03210902411A384A16
:10A3B00055E00120C003E7E70122E369D20393429D
:10A3C0002BD13B0000F0E1F90906090C4D114D4D70
:10A3D0004D274D00FDF756F809E0FDF763F806E05C
:10A3E0000968C90605D4304603E0FDF76BF800287C
:10A3F0003DD0616840004A088018FAF779FE80B2C3
:10A400000146244A103991422BD8511C01400007C3
:10A41000400F084329E01046EBE73B0000F0B5F998
:10A420000906090C2112212121232100FDF72AF818
:10A430000AE0FDF737F807E00968C90606D4304698
:10A4400004E00EE0FDF73EF8002810D061684A08ED
:10A450001018FAF74DFE80B201460E4A10399142AB
:10A4600003D9012503E01046F0E72168C860002009
:10A470006066A0662846F8BD00480040F369FFEF1B
:10A4800000380140401002400044004000093D00F7
:10A49000FFFC0F00EFFF0000F8B5044641654030B7
:10A4A00000262746028380373E602220E06725464B
:10A4B000206F603500281CD01749C162216F1748F2
:10A4C0000863216F16484863206F8663236F606DB1
:10A4D0009C4613462168024660462431FCF7C4F9C5
:10A4E000002806D0102038602E752020A06701209B
:10A4F000F8BD2E7520680168FF220132114301600A
:10A5000020688168012211438160206881684022AF
:10A51000114381600020F8BD79A10008D7A100088F
:10A520002DA10008FFB581B005460F4604466035F1
:10A530000A9E39E0701C37D0FCF73EFB0499401AA4
:10A54000B04222D8002E20D02068016849072BD5C0
:10A55000C069C043000527D401202168C0020862F9
:10A5600020680168FF22A132914301602068816860
:10A570004908490081602020A067E067803420609E
:10A5800000202875032005B0F0BD20680168FF2277
:10A59000A1329143016020688168490849008160C7
:10A5A0002020A067E067EBE72068C1693846884350
:10A5B00005D0002103988142BCD00020E3E70121AF
:10A5C000F8E7000010B50449102009680862024845
:10A5D000FDF738FC10BD0000CC16002001490D200D
:10A5E000887070475400002010B5FEF7AFF9FEF7F1
:10A5F000C7FAC82202490348FDF7D4FD10BD000088
:10A60000200D0020CC160020F8B53E4C0023217808
:10A610003D4A1D46082910D0072947D0062950D0A9
:10A62000052952D0042953D0032954D0002956D0EB
:10A63000012958D002295AD05BE0A17800264A1F90
:10A6400004E0314FBF5DFB189BB2761C9642F8DBED
:10A65000667927799A195118E3786278C9188918A8
:10A66000C9194018C0430006000E1AD1012E14D09B
:10A67000022E16D125482449C018FAF77FFD01F0B3
:10A6800085FF642000F0A6FABFF34F8F21492048D0
:10A69000C860BFF34F8F00BFFDE759081046FFF7B2
:10A6A000B7F92570E570A570A571F8BDA179505472
:10A6B000491CC8B2A071A178491F8842F5D1082071
:10A6C00001E0607007202070F8BDE0700620FAE716
:10A6D00060710520F7E7A070E5700420F3E75528C6
:10A6E00007D10120EFE7AA2803D10220EBE70328D6
:10A6F00003D02570E570A570F8BD0320207020718F
:10A70000F8BD000034010020DE140020E80D002018
:10A710000400FA0500ED00E010B5024A024900F01D
:10A72000E5F910BDD5B80008880100202021020CF1
:10A7300001D010211046020A01D010460839020942
:10A7400001D01046091F820801D01046891E420818
:10A7500001D0881E7047081A7047F8B5040C8BB2F8
:10A76000264682B25E430D0C1046370C5843360421
:10A7700080190021794116466E43370C3604801942
:10A78000794126466E438919F8BD30B47446641E7B
:10A790002578641CAB4200D21D46635D5B00E31864
:10A7A00030BC18474900CA020243100000D0042000
:10A7B0004A0D01D001221043044A490D914201D1B2
:10A7C00002210843012800D105207047FF0700003F
:10A7D0008307FF22DB0E9A408907090E9940002863
:10A7E00008DB830809489B001B181868904308433E
:10A7F000186070470007000F0838830804489B0062
:10A800001B18D86990430843D861704700E400E002
:10A8100000ED00E0BFF34F8F04490348C860BFF369
:10A820004F8F00BFFDE700000400FA0500ED00E0D7
:10A83000F8B504464F1EC8000838211815461E46B4
:10A84000086849683A4606239A4310D02A46334698
:10A85000FAF71AFE3A46D200083AA3181A687F1E81
:10A860005B68FAF75FFD06223B469343EED1022F69
:10A8700023D0042F11D0062F2FD12A463346FAF7C2
:10A8800003FEE36AA26AFAF74DFD2A463346FAF759
:10A89000FBFD636A226AFAF745FD2A463346FAF75A
:10A8A000F3FDE369A269FAF73DFD2A463346FAF75C
:10A8B000EBFD63692269FAF735FD2A463346FAF75C
:10A8C000E3FDE368A268FAF72DFD2A463346FAF75E
:10A8D000DBFD63682268FAF725FDF8BD002210B59C
:10A8E000134610460149FAF737FE10BD0000F03F4D
:10A8F00010B5FAF717FD10BD002210B5134610462B
:10A900001146FAF729FE10BD10B50721024A0020B2
:10A910000907FAF799FE10BD01030000034A10B5BC
:10A9200000201107FAF790FE10BD000001FDFFFFA7
:10A9300002E008C8121F08C1002AFAD17047704708
:10A94000002001E001C1121F002AFBD17047000066
:10A9500001490860704700008C01002008B5002103
:10A96000684601706B46012202212C2000F052FF44
:10A970000221684601706B4601222C2000F04AFF3C
:10A9800008BD000038B504466D20694608706B4666
:10A99000012207492E2000F03DFF0649002C01D07E
:10A9A000054A00E0054A2E2000F01AFF38BD0000DD
:10A9B0000608000006180000070600000716000041
:10A9C00038B504466B4602220021362000F0EEFD29
:10A9D000B3212300FFF7D9FE0E0F08153A3A3A3A91
:10A9E0001C273A3A2F34483A0021684601704078D3
:10A9F0004108490014E06946087880088000401C3E
:10AA000004E06946087880088000801C08701DE01A
:10AA1000684602780A40483202704178802001433B
:10AA20006846417012E0684602780A400270407839
:10AA30004106490EF4E7694648780221084303E0DD
:10AA400069464878FD210840694648706B460122F6
:10AA50000021362000F0DEFE012200AB1146362038
:10AA6000013300F0D7FE38BD69460878CF21084091
:10AA700069462030CAE708B50321684641700121C4
:10AA800001706B4602220021362000F0C3FE012235
:10AA9000D20306212D2000F0A3FE012000F09AF839
:10AAA0000120FFF78DFF08BD08B5020A69464A700C
:10AAB00008706B46022204212D2000F0ABFE03201B
:10AAC000694608706B46012206212D2000F0A2FE87
:10AAD0000020694608706B46012206212D2000F0F7
:10AAE00099FE0A212D2000F047FD08BDF8B5164655
:10AAF0000F460446002503E03946B047641C6D1C30
:10AB000020780028F8D12846F8BD0000F8B54A00A2
:10AB10002B4B520DD6182B4A0C460546142E2BDA19
:10AB2000002E12DA284BFAF7FDFB00221346FAF743
:10AB300053FE40D2002C03DA0124E40700253AE05A
:10AB40002046284337D0214C14E0214F0B46F740D4
:10AB50003B402B4331D01C4BFAF7E4FB0022134659
:10AB6000FAF73AFE27D2002C03DD01200005F04061
:10AB70000419BC4300251EE0332E1EDC334600279B
:10AB8000143BFF43DF40384217D00F4BFAF774FCF9
:10AB900000221346FAF720FE0DD2002C0ADD142EF7
:10ABA0000CD03420811B012088404019A84200D2DB
:10ABB000641C0546BD4321462846F8BD641CF9E7E0
:10ABC00001FCFFFF9C7500883CE4377E0000F03FED
:10ABD000FFFF0F007D2110B5C900484300F001F8C8
:10ABE00010BD002140E000BF00BF00BF00BF00BF9C
:10ABF00000BF00BF00BF00BF00BF00BF00BF00BF5D
:10AC000000BF00BF00BF00BF00BF00BF00BF00BF4C
:10AC100000BF00BF00BF00BF00BF00BF00BF00BF3C
:10AC200000BF00BF00BF00BF00BF00BF00BF00BF2C
:10AC300000BF00BF00BF00BF00BF00BF00BF00BF1C
:10AC400000BF00BF00BF00BF00BF00BF00BF00BF0C
:10AC500000BF00BF00BF00BF00BF00BF00BF00BFFC
:10AC600000BF00BF00BF491C8142BCD37047FFB585
:10AC700081B01E460F46040026D00B99039801436D
:10AC8000A06A3943826807209047002818DB0A9998
:10AC9000A06A3143826806209047002810DB2546D1
:10ACA0002035A979032F01D908200143032E01D9AA
:10ACB00004200143A06A826809209047002806DA30
:10ACC0000120C04305B0F0BD0020C043FAE738467C
:10ACD00000F000F92060304600F0FCF860600A984F
:10ACE00068700398A870EF702E710B98687100203F
:10ACF000E8E70000F7B50446002090B0009001900E
:10AD0000002C05D06A46062101F07AFC062803DAF9
:10AD10000020C04313B0F0BD684640780102684689
:10AD2000007800040918684680780818FAF7C8FC0B
:10AD3000054668460391007901026846C078000420
:10AD40000918684640790818FAF7BAFC0322064643
:10AD50000F4692075C4BFAF73FFD07D200225B4B90
:10AD600030463946FAF782FB06460F460322920721
:10AD7000554B28460399FAF72FFD07D20022534B73
:10AD800028460399FAF772FB054603912068FAF703
:10AD900097FC02460B4630463946FAF7DDFB07467C
:10ADA0000A200791205EFAF777FC3A46079BFAF7EC
:10ADB0006BFB064608200991205EFAF75BFC002138
:10ADC000C943FAF7A3FAFAF7DFFC3246099BFAF710
:10ADD000A9FA069108906068FAF772FC02460B46E1
:10ADE00028460399FAF7B8FB05461A200E46205E5E
:10ADF000FAF752FC2A463346FAF746FB0C900991C3
:10AE00001620205EFAF748FC099B0C9AFAF78AFA9A
:10AE100005910A902A46334638460799FAF734FBDB
:10AE2000059B0A9AFAF730FB05910A901420205EE0
:10AE3000FAF732FC3A46079BFAF726FB07461C2036
:10AE40000791205EFAF728FC2A463346FAF71CFBE6
:10AE50000E900B911820205EFAF71EFC0B9B0E9AA9
:10AE6000FAF760FA2A463346FAF70EFB0B910E907A
:10AE70002069FAF711FC0B9B0E9AFAF753FA2A464F
:10AE80003346FAF701FB05460E46E068FAF704FC84
:10AE90002A463346FAF746FA3A46079BFAF742FA49
:10AEA000059B0A9AFAF73EFA01229207084BFAF735
:10AEB000EBFA02460B46129C0898069903C41198B7
:10AEC0000CC0002026E70000FFFF5F41000070413A
:10AED000E17A843F00B50121C9040300FFF755FC66
:10AEE000081A05080B0E1114171A0320C00400BD20
:10AEF0000720C00400BD0F20C00400BD1F20400378
:10AF000000BD3F20400300BD7F20400300BDFF2067
:10AF1000400300BD084600BDFEB5264F0D460400A7
:10AF20000FD0002D0DD0264600202036B071F071D4
:10AF300029680D208847002801DA7800FEBD102816
:10AF400001D03846FEBDA562E968002901D028205D
:10AF50008847204600F030F80028F3DBA06AA521DE
:10AF600082680E209047A06A962182680F20904741
:10AF7000A06A0221826862209047A06A002182684C
:10AF80000E209047A06A002182680F2090477179B7
:10AF90003020019100900623202201212046FFF756
:10AFA00066FE0028CEDB204600F0AEF80028C9DBA4
:10AFB0000020FEBDFFFFFFFF10B586B00446142140
:10AFC0006846FAF7F4F8002C7ED0A06A1221436894
:10AFD0006A4610209847122877D1684600780122E7
:10AFE000010168464078120300090818434920818E
:10AFF000884201DD801A2081684683784078000706
:10B00000000D18186081884201DD801A6081684651
:10B010000079012201016846C07812050003091871
:10B0200068464079000908183549E060884201DD2A
:10B03000801AE060684640790007030B6846807913
:10B0400000021B186846C07918182061884201DD8B
:10B05000801A20616846417A007A0002081802B21C
:10B06000284801210904A282824201DD521AA282EB
:10B070006A46D37A927A12029A1812B2E282824215
:10B0800001DD521AE2826A46537B127B12029A1841
:10B0900012B22283824201DD521A22836A46D37B96
:10B0A000927B12029A1812B26283824201DD521A16
:10B0B00062836A46537C127C12029A1812B2A283EF
:10B0C000824204DD501A01E00BE008E0A083A06A90
:10B0D000016828208847002806DA0120C04306B00E
:10B0E00010BD0020C043FAE7C011C007203400287B
:10B0F00000D0802060710020F1E70000FF07000011
:10B10000FFFF0700FF7F000010B5040009D0A06A10
:10B110000721826808209047002805DA0120C043F3
:10B1200010BD0020C04310BD072020342070002037
:10B1300010BD0000FEB5044600200190009060792B
:10B14000734940000E5A61782578491E7148CFB284
:10B150000163042D77D0072D75D00021029121784D
:10B1600001736C49E379012292058969002B6CD047
:10B17000914381616748217A4173217A8269890705
:10B18000890B0A4382610021042000F034FB32461F
:10B1900061492E2000F024FB3846FFF7F3FB5F4E99
:10B1A0000522705D810040185D49431807212B205E
:10B1B00000F030FB5B49029801220B180B2128207C
:10B1C00000F028FB705D584980000A580C212820A7
:10B1D00000F011FBE079554980004018A179490041
:10B1E000425A0221272000F0FBFA51487E00825B80
:10B1F0000421272000F0F4FAE079002829D0A07873
:10B2000004282CD0282069460872202206212720F5
:10B2100000F0E6FA02AB01222621272000F0FAFA1C
:10B22000444938014018E178890042580821272014
:10B2300000F0E1FAA17A601C627A0902114313D08E
:10B2400016E000E001E0012188E71143F608816182
:10B2500090E764220621272000F0C2FAE0E71020E0
:10B26000694608720246D1E733490172090A417200
:10B27000417A007A0A0202432021272000F0B0FA26
:10B280002E4F0C2123203A6800F0B5FAF01982887D
:10B290000421232000F0A4FAA07900280BD0E07943
:10B2A0002749012243180021212000F0B3FA03208E
:10B2B0000190012000902A07120F100102436078CC
:10B2C00000218007000B024301980005024300980B
:10B2D000400402432079C006400902436079C00659
:10B2E00002431F2000F087FAA07861780123084309
:10B2F00002040848DB030261E179490319430A4368
:10B3000002610021082000F076FA0020FEBD000056
:10B3100034C70008BC01002004280000DCC6000877
:10B320002400002042000020E4C6000804C70008F2
:10B3300010C7000814C7000841100000FCC6000830
:10B340004400002038B50C4607498A8B002102438F
:10B350002C2000F045FA684604706B460122062155
:10B360002C2000F057FA38BDBC01002010B5FFF7C3
:10B37000F5FA10BD10B504460421362000F0FCF8A3
:10B380000121C902002C01D0084300E08843024695
:10B390000421362000F02FFA10BD000038B54020FF
:10B3A0006946087000210E2000F0E6F804460022ED
:10B3B00011460E2000F01FFA6B46012200210D20DD
:10B3C00000F028FA074A00210F2000F014FA00F0DC
:10B3D000EDF9224600210E2000F00DFA024800216E
:10B3E000017338BDF8FF2724DC010020FEB50546B7
:10B3F000042069460870514C0020607521462031B8
:10B40000206348710873A0836063A06300F0C8F8EC
:10B410004B4E206002E000F0C3F82060B042FAD149
:10B420000020FFF7CDFA00F0BBF8464E20603078E0
:10B43000242801D9243806E00621F9F759FE06220E
:10B44000101A40010843020601040A4301020A439C
:10B450000243B260706000211E2000F0CCF900F0C1
:10B460009FF820606B4601220021242000F0D2F9D1
:10B470001E20FFF719FB86B2300AA0730420FFF7E5
:10B4800013FB074600F08CF820603806000E0DD044
:10B4900002206946087101AB012212212D2000F023
:10B4A000B9F9A08B012109030843A08300F078F8C3
:10B4B00020600620FFF7F8FA60600720FFF7F4FA33
:10B4C000A060F006C00E207501D110202075C0B21A
:10B4D00000F0DCF9E80707D0FFF7CDFAA08B0121D7
:10B4E000C9020843A0830AE00521362000F02EF8A7
:10B4F0001549084002460521362000F071F9012067
:10B50000FFF75EFA0021042000F036F8A061002168
:10B51000262000F031F81521890308430246002156
:10B52000262000F068F900222621362000F058F984
:10B5300000F036F820600020FEBD0000BC010020B5
:10B540003001CADE18000020FFFD000038B5094CAC
:10B5500089B280B26B46022200F028F8002806D19A
:10B5600068464078010268460078081884B2204690
:10B5700038BD0000FFFF000038B50024E44389B265
:10B5800080B26B46042200F011F8002806D1032196
:10B590006846435C2202D418491EFAD5204638BDBD
:10B5A00010B500210846FFF7E7FF10BD38B50029A8
:10B5B00009D0402420436C462070C8B27F2906D8A9
:10B5C000607002200AE069460870012006E08024CD
:10B5D00020436C466070C809A0700320694600F0E3
:10B5E000AFFF38BD10B5144603460A462146112068
:10B5F000FFF7DCFF10BD10B5034605220021152022
:10B60000FFF7D4FF10BD10B5034605220021172017
:10B61000FFF7CCFF10BD38B505460020694608701D
:10B6200000F0C4F8FF2401342246002D01D003228B
:10B63000120200210D2000F0D3F8002D13D06B462C
:10B64000012203210F20FFF7B1FF684600780007B1
:10B6500009D5FFF7A3FE224600210D2000F0C0F817
:10B660000020C04338BD002038BD10B5024601217E
:10B670000A2000F0C0F810BD10B5044600211A20C1
:10B68000FFF77AFF000D22030005120B0243002191
:10B690001A2000F0B0F810BD10B5024602492E2065
:10B6A00000F09EF810BD000004180000F8B5054633
:10B6B0006B46012203210420FFF778FF0126114C7D
:10B6C0003607002D0DD02A4600210C2000F088F806
:10B6D000694608781021084369460870A06930431C
:10B6E00007E069460878EF21084069460870A069BC
:10B6F000B0430B46A06101220321042000F08AF828
:10B70000F8BD0000BC01002010B502460021182041
:10B7100000F066F810BD0000F8B507460025684641
:10B720000570B807204C2E4600280ADA80206946AA
:10B7300008706B46012200210D2000F06BF80120FB
:10B740002073F8076946087821D006210843694626
:10B7500008706B46012200210D2000F05BF80321E8
:10B760000F20FFF7F3FE8121C900084219D04020C5
:10B77000694608706B46012200210D2000F04AF84E
:10B780000020FFF7F7FD00252673ED4309E00221B5
:10B790000843694608706B46012200210D2000F025
:10B7A00039F82846F8BD0000DC0100201CB56B46C6
:10B7B000012203210F20FFF7F9FE6846007840229E
:10B7C000C1091040C9014000814208D001206946EA
:10B7D0000871024601AB03210D2000F01BF81CBDCF
:10B7E00008B56B461A70120A5A7089B280B20222EA
:10B7F00000F010F808BD38B500236C46E254120A78
:10B800005B1C042BFADB89B280B22346042200F0D1
:10B8100001F838BD38B58024002909D0C025284357
:10B820006D462870C8B27F2907D86870022009E0E9
:10B83000204369460870012004E020436870C8096D
:10B84000A8700320694600F025FF38BD10B51446E6
:10B85000012312189B029A4202D90020C04310BD56
:10B860000B46821E21460920FFF7D4FF002010BDA1
:10B8700010B5054A8905126901430A4300210820D1
:10B88000FFF7B9FF002010BDBC01002038B5044609
:10B890006B4601220E212B20FFF788FE68460078B8
:10B8A000E10640094001C90E0143684601706B463C
:10B8B00001220E212B20FFF7ADFF38BD10B500216E
:10B8C00042541C06120A22431B0A491C0429F7DBB6
:10B8D00010BD000013B501231A4669460248FCF763
:10B8E00093FC00981CBD0000CC1600207CB5002401
:10B8F00025466846FFF77FFE04206946220E2D028A
:10B90000154322020C5C1443401EF7D520462946FD
:10B910007CBD7CB5002425466846FFF774FE0420F4
:10B920006946220E2D02154322020C5C1443401E70
:10B93000F7D5204629467CBDFBF74CF9FEF708F900
:10B94000FDF718F83D493E48002522C00560856195
:10B95000C5613C490562C1600838FBF7CDFAFCF7C8
:10B96000F5FFFDF70DF9FDF7A9F8FCF7BBFF05247E
:10B9700001222407D1032046FBF717F9FDF79AFEB1
:10B98000FCF7A8FEFAF70AF9FAF78CF9FAF75AF970
:10B99000FCF7BCFC0721A015FFF7D4FCFFF7E6FC81
:10B9A000012211032046FBF700F92548C822264949
:10B9B000C830FCF7F7FB254F254E264C3878002879
:10B9C0000FD13078002801D003280AD10121C90203
:10B9D0002148FBF7DDF8002803D101210846FBF7D9
:10B9E0009FFBE078002826D06078002823D0E570FF
:10B9F00020780F280AD90120174900038861FEF733
:10BA0000F5F901201449000388620CE0012251037A
:10BA10001148FBF7CAF8FEF7E9F9012100224903B2
:10BA20000D48FBF7C2F8FCF77BFD208C0028C5D041
:10BA3000401E2084C2E7FCF773FDBFE7007C004096
:10BA400004160020FFFF0000200D00205A000020F7
:10BA5000810000203C0100200004005010B586B099
:10BA60001748FBF7CCF914216846F9F7A0FB1548F5
:10BA700000900320019000200290052069460007F5
:10BA8000FAF7CAFF69461048FAF7C6FF69460F4839
:10BA9000FAF7C2FF01210846FBF742FBFF240134FD
:10BAA0002046FBF715FB0A4908680422104308608A
:10BAB0002046FBF71DFBFBF723FB06B010BD000083
:10BAC00004160020FFFF0000000400500008005092
:10BAD0000070004010B50122920217491748FAF78A
:10BAE00063F91548164902888A4223D0018004214F
:10BAF0008180FF21F531C1800A21018100211E22B0
:10BB00004181D24382810122C28181834323C38642
:10BB100002230387782343878287C2870246403205
:10BB2000118451849184C183918014238382118272
:10BB300000F02CFD10BD0000E80D002000FC000806
:10BB4000AA550000F0B51FB496B084460C460246D4
:10BB5000199D18980390490068006300490840083F
:10BB60000193002A01D0012600E000269E19FE4B19
:10BB7000F6185B109E422BD36E00039F0296002F97
:10BB800000D00127F719F84EF84BBE199E421FD37B
:10BB9000039E0346F64F334309D03B469C4201D1F6
:10BBA000002A04D0019B002A05D0012604E00020D1
:10BBB00039461BB0F0BD00269E19EE4B9E4207D8B9
:10BBC000039F029E002F00D00127F6199E4207D93D
:10BBD0002B4660462146189AFEF78AFE1BB0F0BD40
:10BBE0000023002C29DAE44EB04226DAE34EB042BC
:10BBF00001DB022321E0DE4EB0421EDBE04E070DEA
:10BC0000BE19142E09DD3427BF1B039EFE4001968A
:10BC1000BE40039FBE420BD00FE0039F002F0CD10C
:10BC20001427BF1B0646FE400196BE40864204D143
:10BC3000019BDE07F60F02239B1B0E46164318D10D
:10BC4000002D16DA002C03D0022B01D0012B06D0D8
:10BC50000220FEF77DFEFEF741FE1BB0F0BD022084
:10BC6000FEF776FEFEF73AFE0122D20751401BB0E6
:10BC7000F0BD039E002E61D1BF4EB04220D1C1481D
:10BC8000844201D1002A08D0B948814209DB002D45
:10BC900010DB189829461BB0F0BD0020B4491BB03A
:10BCA000F0BD002D06DA01222946D207189851402E
:10BCB0001BB0F0BDB4497944086849681BB0F0BDB9
:10BCC000AB4FB84225D1002D1FDA002904D0B14274
:10BCD00012D1002A09D018E0002A72D1A649E20F39
:10BCE0000020D20711431BB0F0BD0020E20F014637
:10BCF000D20711431BB0F0BDB14206DA2346002043
:10BD00003946F9F729FC1BB0F0BD104621461BB09F
:10BD1000F0BDB14212DA0126B607B54203D123467F
:10BD200010461946FEE3994EB54207D1261E05DBA3
:10BD30001046314600F040FC1BB0F0BD67007F08A4
:10BD40001646002A40D100290AD08B4A914229D1B7
:10BD5000002C0EDD002D1CDB002011461BB0F0BDB9
:10BD6000022B16D0002C14D0012B12D1002C14DB86
:10BD70000FE0002C28DA002D09DB012B03D0002076
:10BD80007D491BB0F0BD002081491BB0F0BD012BE7
:10BD900003D0002001461BB0F0BD00200121C907DF
:10BDA0001BB0F0BD724A91420ED1002C01DA002B7B
:10BDB00017D0022B06D00020C043F9F76DFC1BB052
:10BDC000F0BD90E20120F8E7E217521C94461A43B6
:10BDD00007D000220892664C62465B1E1A4307D0C9
:10BDE00009E00120FEF7B4FDFEF786FD1BB0F0BDB3
:10BDF0000022644C0892674A90427DDD664B674A98
:10BE000098421FDD914202DC002D05DB4DE05848D1
:10BE1000814217DB002D48DD0220FEF799FDFEF779
:10BE200073FD05460E460022534B21460898F9F74C
:10BE30002BFB084671004908C00FC0070143284684
:10BE40001BB0F0BD914215DA002D2EDA0220FEF76C
:10BE50007FFDFEF759FD05460E460022464B214662
:10BE60000898F9F711FB72005208C80FC007024387
:10BE7000114617E03E4B994223DD002D15DD0220CF
:10BE8000FEF766FDFEF740FD05460E4600223A4BE2
:10BE900021460898F9F7F8FA084671004908C00FDA
:10BEA000C007014328461BB0F0BD0220FEF750FD3D
:10BEB000FEF734FD49004908E20FD20711431BB0D9
:10BEC000F0BD002230463946F9F7D0FA0122054686
:10BED0000E46D243F9F7B8FB314A324BF9F7CCFAA8
:10BEE0002A463346F9F7D0FA0022284BF9F7C4FA6C
:10BEF00007462A46334600E064E00391104619469F
:10BF0000F9F7C2FA3A46039BF9F7BEFA074603224D
:10BF100009915207244B28463146F9F7B5FA0791A3
:10BF20000C90224A204B38460999F9F7ADFA07469A
:10BF300001911F4A1F4B28463146F9F7A5FA3A46A8
:10BF4000019BF9F793FA07460B46024609910799B8
:10BF50000C98F9F7E7F900250E462846079B0C9A3E
:10BF6000F9F784FA3A4627E0FFFF1F00FFFF0F00B2
:10BF70000000F03F0000E0FF0000F07F00004043C1
:10BF800001FCFFFF0000F0BF560B00000000E03F87
:10BF90000000F0FF0000E0410000F043FFFFEF3F32
:10BFA000555555555555D53F4715F73FFE822B65DD
:10BFB00044DF5DF80BAE543E099BF9F75DFA02468B
:10BFC0000B4652E1012500202D05A94207DA352252
:10BFD00030463946F9F738FB06463420C0430A1587
:10BFE0001218FE48101803900803FD49000B014386
:10BFF0000F46FC49884201DC002003E0FA498842F0
:10C0000002DA0120119005E0002011900398401CF5
:10C010007F1B039011980597C200F4480F92784453
:10C02000801843680268394630460D930292F9F74A
:10C030001DFA07910C9030460D9B029A0599F9F76D
:10C0400071F902460B460020E549F9F785FA099196
:10C050000490079B0C9AF9F717FA129000201090A1
:10C06000E3480D46784400680E9001217810490796
:10C07000084311990D9B890440180121C9044718F0
:10C080003946029A0E98F9F7F1F93246059BF9F70D
:10C09000F3F902460B4629461098F9F7F5F90646DA
:10C0A00002913B4629460E9A1098F9F7EDF9079B45
:10C0B0000C9AF9F7E1F93246029BF9F7D7F9099B97
:10C0C000049AF9F7E1F90591129A0A902B46104665
:10C0D0001946F9F7D9F906460246C6480F460B46F7
:10C0E00006217844FEF7A4FB32463B4600910490BB
:10C0F00010461946F9F7C8F9009B049AF9F7C4F9F4
:10C1000006460F462B461946129A1098F9F70AF977
:10C11000059B0A9AF9F7B8F932463B46F9F702F956
:10C12000109A079104902B4610461946F9F7ACF97E
:10C13000B14E0022334609910290F9F7F3F8079BBC
:10C14000049AF9F7EFF800200746024633460091BB
:10C15000F9F78CF9099B029AF9F788F9079B049A79
:10C16000F9F78AF906460D913A462946009B109840
:10C17000F9F78AF907910C902B463046129A0D99DF
:10C18000F9F782F905460E463A46009B05990A984A
:10C19000F9F77AF933462A46F9F7C4F802460B460E
:10C1A0000746099107990C98F9F7BCF800250E4647
:10C1B0002846079B0C9AF9F759F93A46099BF9F773
:10C1C0005BF907460722099152078C4B31462846F6
:10C1D000F9F75AF907910090894A884B384609992E
:10C1E000F9F752F907460191864A874B31462846AE
:10C1F000F9F74AF93A46019BF9F794F8834B7B44E7
:10C200000F9A9B181A685B68F9F78CF802900991ED
:10C210000398F9F741FA05910490099B029A07994E
:10C220000098F9F77FF87A4B7B440F9A9B181A68AD
:10C230005B6817460393F9F775F8059B049AF9F7BD
:10C2400071F80E462846059B049AF9F70FF93A460D
:10C25000039BF9F70BF9079B009AF9F707F9099B7C
:10C26000029AF9F709F902460B46199900200C9039
:10C270000F461898F9F708F9029104903B460C9A7A
:10C2800019991898F9F7F2F82A463346F9F7FCF8A5
:10C29000029B049AF9F746F809910E902A46334614
:10C2A00039460C98F9F7F0F806460F46099B0E9AA6
:10C2B000F9F738F8574A0D46914220DB5242AA1846
:10C2C000024310D132463B46F9F7D0F8049003916F
:10C2D000514A524B09990E98F9F724F8039B049A96
:10C2E000F9F77AFA1ED20220FEF732FBFEF70CFBBA
:10C2F00049004908E20FD20711431BB0F0BD6A00A4
:10C30000474B52089A420DD3464AAA18024300D01E
:10C31000CBE532463B46F9F7A9F8099B0E9AF9F7A7
:10C320005BFAF5D96800002340082C490393020DFD
:10C330003D4B5218984223DD01200005521CD0408D
:10C3400042195000400D4018384979440968134695
:10C350008C463749C1408B4312030121120B09055A
:10C3600051181422101AC1400391002D01DA4842DD
:10C370000390624630463946F9F778F806460F468C
:10C3800032463B4609990E98F8F7CCFF00252A461D
:10C39000284B28460591F9F777F807910C90264A23
:10C3A000264B28460599F9F76FF80091029032461E
:10C3B0003B4628460599F9F759F8099B0E9AF9F773
:10C3C0005BF81F4A1F4BF9F75FF8009B029AF8F7DA
:10C3D000A9FF07460B460246099135E001FCFFFF25
:10C3E0000000F03F8E9803007AB60B00660700004D
:10C3F000A8070000D20600000000084009C7EE3F71
:10C40000FD033ADCF5015B14E02F3EBEA6050000FB
:10C410006C05000000009040FE822B654715973C9C
:10C4200000CC904000346F3F0000E03FC2040000A9
:10C43000FFFF0F00432EE63F396CA80C615C20BE65
:10C44000EF39FAFE422EE63F07990C98F8F76AFF9B
:10C4500005460E46079B0C9AF9F708F83A46099BE1
:10C46000F9F70AF809912A4633460E901046194604
:10C47000F9F70AF8074602462F480B4605910521B1
:10C480007844FEF7D5F93A46059BF8F7FDFF2A46B2
:10C490003346F8F7F1FF0746019128463146099BDC
:10C4A0000E9AF8F7F1FF099B0E9AF8F73BFF01236C
:10C4B00004910C9000229B0738460199F8F7D6FFAB
:10C4C00005910E903A4628463146019BF8F7DCFF6D
:10C4D000059B0E9AF9F740F8049B0C9AF8F7C6FFF3
:10C4E0002A463346F8F7C2FF0022144BF8F7C4FF80
:10C4F000064603980D46000541190915002912DC6E
:10C5000030462946039AF9F79FF8FEF74BF90428BD
:10C5100001D1FEF703FA30462946039AF9F794F859
:10C52000064601E004E029180B46324621460898E9
:10C53000F8F7AAFF1BB0F0BD640300000000F03F55
:10C54000F0B58C4600251026052109078E620E4C99
:10C5500008E067467F5DE760A768FF07FCD0E768F3
:10C560001F706D1C8542F4DB0020074606E0E76083
:10C57000A568ED07FCD0E5681D54401C9042F6D339
:10C580008E610020F0BD00000030014070B572B631
:10C590000124074DA40221462846F9F7EBFB0028A9
:10C5A00004D0224603492846F9F788FC62B670BDDC
:10C5B00000FC0008E80D0020F8B506460C46F9F727
:10C5C00019FA051E0F4600D00120014349000B480F
:10C5D0004908411AC90F0DD0002E01D0012100E0F9
:10C5E00000210C4361004908401AC00F02D101200C
:10C5F000FEF7AEF928463946F8BD00000000F07F8E
:10C60000F8B515460E460746002407E03819C0B2B3
:10C6100000F008F8641C2870E4B26D1CB442F5D335
:10C620003046F8BD10B50446FBF716FFEE20FBF7C9
:10C63000E6FEFBF74AFF2046FBF7E1FEFBF745FF6E
:10C64000FBF70AFFEF20FBF7DAFEFBF73EFF0020C7
:10C65000FBF7A8FE0446FBF71AFF204610BD704703
:10C6600070B50D460446FBF7F7FEEE20FBF7C7FE5C
:10C67000FBF72BFF2046FBF7C2FEFBF726FF284601
:10C68000FBF7BDFEFBF721FFFBF701FF0A20FEF7DA
:10C69000A8FA70BDF0B50025102605279C463F0777
:10C6A0000B46BE620C4C06E0595DE160A168C9070B
:10C6B000FCD0E1686D1C8542F6DB002007E0614696
:10C6C000095CE160A168C907FCD0E168401C9042A8
:10C6D000F5D3BE610020F0BD003001400000010232
:10C6E00003040005405C0000A05C0400C06C08006E
:10C6F000805C0400E03F1E00E07D1E0007A90225CB
:10C7000070889B880A0016000100060001000200E4
:10C7100087008D002D001A3152001A339A001A3505
:10C720001D011A376B003B31BE003B335E013B35C8
:10C7300096023B37000099599959EB518F421E459B
:10C74000142E0080EB51F5283333E13A703DE13A85
:10C75000C235852BC2353333C235C235AE47E13AD7
:10C760005138A330513800000000000000000102E1
:10C77000030406070809030406080C1018203000FB
:10C780000000000102030400000000000000F03F70
:10C79000000000000000F83F000000000000000062
:10C7A0000000004003B8E23F00000000000000006D
:10C7B00006D0CF43EBFD4C3E033333333333E33FFB
:10C7C000FFAB6FDBB66DDB3F4D268F515555D53F27
:10C7D00001411DA96074D13F65DBC9934A86CD3FF5
:10C7E000EF4E454A287ECA3F3E5555555555C53FE3
:10C7F00093BDBE166CC166BF2CDE25AF6A56113FD5
:10C80000F16BD2C541BDBBBED0A4BE726937663ED6
:10C81000000000000000000038C8000800000020F0
:10C8200090010000BC5A00089CC80008900100203C
:10C83000681A000040A900080124130704380D09F4
:10C840001E080540082609104008560A131D043B1F
:10C8500008BE0516D8BC40100852010338C842056E
:10C86000740CE5A00F1B0202DD140901022281F005
:10C870001F66810498899686967982159803981484
:10C8800098879674977882439788967197778249AC
:0CC89000F10139293F92049220000000C1
:04000005080050C1DE
:00000001FF
